:100000000C9480170C949D170C949D170C949D17BD
:100010000C949D170C949D170C949D170C949D1790
:100020000C949D170C949D170C949D170C949D1780
:100030000C949D170C94E7320C949D170C949D170B
:100040000C949D170C949D170C949D170C949D1760
:100050000C949D170C949D170C949D170C949D1750
:100060000C949D170C949D170C949D170C949D1740
:10007000FFFFFFFFFFFFFFFFFFFFFFFFFFFFFFFF90
:10008000FFFF00FFFF2030FFFFFF0111102131FFB4
:10009000FF030212223332FFFF700413242334FFC4
:1000A000FF737464145444FFFFFF7263534342FFB1
:1000B000FFFF6252514041FFFF71FF61FF50FFFFA0
:1000C000FFFFFFFFFFFFFFFFFFFF60FFFFFFFFFFDF
:1000D000FFFFFFFFFFFFFFFFFFFFFFFFFFFFFFFF30
:1000E000FFFFFFFFFFFFFFFFFFFFFFFFFFFFFFFF20
:1000F00044000004000404000004040004000004A0
:1001000000040400040000040400000400040400CF
:1001100000040400040000040400000400040400BF
:1001200004000004000404000004040004000004AF
:10013000000404000400000404000004000404009F
:10014000040000040004040000040400040000048F
:10015000040000040004040000040400040000047F
:10016000000404000400000404000004000404006F
:10017000808484808480808484808084808484805F
:10018000848080848084848080848480848080844F
:10019000848080848084848080848480848080843F
:1001A000808484808480808484808084808484802F
:1001B000848080848084848080848480848080841F
:1001C000808484808480808484808084808484800F
:1001D00080848480848080848480808480848480FF
:1001E00084808084808484808084848084808084EF
:1001F00000000000000000000000000000000000FF
:10020000000000B441B541CD443B45CE44EA440032
:1002100000ED44ED44205D4000020000FFFF003788
:10022000B441FEFF0100006B0C478738E60000BCBC
:10023000211840001A1C27343227373A331B350067
:1002400000000000000000000000000000000000AE
:100250000000007600000000000000000000842084
:10026000000000808080808080889691900000004F
:100270000000000000012101EA8096922121A901DD
:100280000007CDF50811C0013E80D71B7AB320F8D6
:1002900006203E8AD710FDED5B33402A32401922FA
:1002A00032407CE607C60D47C5CDF5083A3240E638
:1002B00007C604D7C178FE1428030418EB79FE1F83
:1002C00028030C18D2010008C5CDF50811824001A1
:1002D0000600CD6B0B2A10401121002BE57EFEA9F4
:1002E000200E237EFE7628FAFE802829E1C38D4168
:1002F000FE92201E3680237EFE7628FAFE8A281281
:10030000197EFE80280AFE8A28083680197E18F693
:100310003692E118C6E106040B78B120FB3A3E4064
:100320003C323E40CB4720AD3A3C403D28363A2552
:10033000403C2830197EFE80280AFE8A2808368034
:10034000197E18F636922186407EFE1C2005362541
:100350002B18F63D77FE1C200B2B7EFE1C20053E45
:1003600001323C40C10C79FE1A200778FE14281F88
:100370001807FE2020030E000479E601C69632839A
:1003800040C3D140C1CDF50806063E97D710FD3ECB
:1003900021328540328640C976000A0E00F9D41D0C
:1003A00022211E1C7E8F01100000767600000000C6
:1003B000000000000000000000000000000000003D
:1003C00000000000000000000000000076000000B7
:1003D000000000000000000000000000000000001D
:1003E0000000000000000000000000000076000097
:1003F00000000000000000000000000000000000FD
:100400000000000000000000000000000000760076
:1004100000000000000000000000000000000000DC
:100420000000000000000000000000000000007656
:1004300000000000000000000000000000000000BC
:1004400000000000000000000000000000000000AC
:100450007600000000000000000000000000000026
:10046000000000000000000000000000000000008C
:100470000076000000000000000000000000000006
:10048000000000000000000000000000000000006C
:1004900000007600000000000000000000000000E6
:1004A000000000000000000000000000000000004C
:1004B00000000076000000000000000000000000C6
:1004C000000000000000000000000000000000002C
:1004D00000000000760000000000000000000000A6
:1004E000000000000000000000000000000000000C
:1004F0000000000000760000000000000000000086
:1005000000000000000000000000000000000000EB
:100510000000000000007600000000000000000065
:1005200000000000000000000000000000000000CB
:100530000000000000000076000000000000000045
:1005400000000000000000000000000000000000AB
:100550000000000000000000760000000000000025
:10056000000000000000000000000000000000008B
:100570000000000000000000007600000000000005
:10058000000000000000000000000000000000006B
:1005900000000000000000000000760000000000E5
:1005A000000000000000000000000000000000004B
:1005B00000000000000000000000007600000000C5
:1005C000000000000000000000000000000000002B
:1005D00000000000000000000000000076000000A5
:1005E000000000000000000000000000000000000B
:1005F0000000000000000000000000000076000085
:1006000000000000000000000000000000000000EA
:100610000000000000000000000000000000760064
:1006200000000000000000000000000000000000CA
:100630000000000000000000000000000000007644
:1006400000000000000000000000000000000000AA
:10065000000000000000000000000000000000009A
:100660007600000000000000000000000000000014
:10067000000000000000000000000000000000007A
:1006800000760000000000000000000000000000F4
:10069000000000000000000000000000000000005A
:1006A00000007600000000000000000000000000D4
:1006B000000000000000000000000000000000003A
:1006C0000000007680F5D4241D251E7E8E000000DB
:1006D00000190B38263B2A0E350E27343227373ABD
:1006E000330E0B768E0000000000000000000000BA
:1006F00000000000000000000000000000000000FA
:10070000FF0FF000FF0FF00055FF55FFFFFFFFFF49
:10071000FFFFFFFFFFFFFFFFFFFFFFFFFFFFFFFFE9
:10072000FFFFFFFFFFFFFFFFFFFFFFFFFFFFFFFFD9
:10073000FFFFFFFFFFFFFFFFFFFFFFFFFFFFFFFFC9
:1007400000000000000000000000000000000000A9
:100750000000000000000000000000000000000099
:100760000000000000000000000000000000000089
:100770000000000000000000000000000000000079
:1007800000F00FFF00F00FFFAA00AA000000000019
:100790000000000000000000000000000000000059
:1007A0000000000000000000000000000000000049
:1007B0000000000000000000000000000000000039
:1007C0000000000000000000000000000000000029
:1007D0000000000000000000000000000000000019
:1007E0000000000000000000000000000000000009
:1007F00000000000000000000000000000000000F9
:10080000FF0FF000FF0FF000AAFFAADBE3F7FFC322
:10081000FBDFFFFFFFFFFFFFFFFFFFFFC3E7C3C3D8
:10082000F781C381C3C3C383C3878181C3BDC1FDB6
:10083000BBBFBDBDC383C383C301BDBDBDBD7D8182
:1008400000000000000000000000000000000000A8
:100850000000000000000000000000000000000098
:100860000000000000000000000000000000000088
:100870000000000000000000000000000000000078
:1008800000F00FFF00F00FFF550055241C08003C3E
:100890000420000000000000000000003C183C3C68
:1008A000087E3C7E3C3C3C7C3C787E7E3C423E026A
:1008B000444042423C7C3C7C3CFE42424242827E7E
:1008C0000000000000000000000000000000000028
:1008D0000000000000000000000000000000000018
:1008E0000000000000000000000000000000000008
:1008F00000000000000000000000000000000000F8
:10090000FF0FF000FF0FF00055FF55DBDDC1FFBD0D
:10091000F7EFEFFBFFF7FFEBFDEFFFFFB9D7BDBD33
:10092000E7BFBFFDBDBDBDBDBDBBBFBFBDBDF7FD0D
:10093000B7BF999DBDBDBDBDBFEFBDBDBDDBBBFBA1
:1009400000000000000000000000000000000000A7
:100950000000000000000000000000000000000097
:100960000000000000000000000000000000000087
:100970000000000000000000000000000000000077
:1009800000F00FFF00F00FFFAA00AA24223E004251
:10099000081010040008001402100000462842420B
:1009A0001840400242424242424440404242080211
:1009B000484066624242424240104242422444045D
:1009C0000000000000000000000000000000000027
:1009D0000000000000000000000000000000000017
:1009E0000000000000000000000000000000000007
:1009F00000000000000000000000000000000000F7
:100A0000FF0FF000FF0FF000AAFFAAFF87D7EFFB50
:100A1000F7EFF7F7C1F7FFF7FBFFFFFFB5F7FDF3C0
:100A2000D78383FBC3BDBD83BFBD8383BF81F7FD78
:100A30008FBFA5ADBDBDBDBDC3EFBDBDBDE7D7F784
:100A400000000000000000000000000000000000A6
:100A50000000000000000000000000000000000096
:100A60000000000000000000000000000000000086
:100A70000000000000000000000000000000000076
:100A800000F00FFF00F00FFF55005500782810040C
:100A9000081008083E080008040000004A08020C7C
:100AA000287C7C043C42427C40427C7C407E0802A4
:100AB00070405A52424242423C1042424218280878
:100AC0000000000000000000000000000000000026
:100AD0000000000000000000000000000000000016
:100AE0000000000000000000000000000000000006
:100AF00000000000000000000000000000000000F6
:100B0000FFFFFFFF0F0F0F0F5555FFFFDFC1FFF76F
:100B1000F7EFFBEFFFC1C1C1F7FFFFFFADF7C3FD6B
:100B2000B7FDBDF7BDC181BDBFBDBFBFB1BDF7BD85
:100B3000B7BFBDB5BD83AD83FDEFBDBDBDE7EFEF75
:100B400000000000000000000000000000000000A5
:100B50000000000000000000000000000000000095
:100B60000000000000000000000000000000000085
:100B70000000000000000000000000000000000075
:100B800000000000F0F0F0F0AAAA0000203E0008EB
:100B900008100410003E3E3E0800000052083C02CF
:100BA00048024208423E7E42404240404E42084295
:100BB0004840424A427C527C021042424218101085
:100BC0000000000000000000000000000000000025
:100BD0000000000000000000000000000000000015
:100BE0000000000000000000000000000000000005
:100BF00000000000000000000000000000000000F5
:100C0000FFFFFFFF0F0F0F0FAAAAFFFFDFF5FFFF88
:100C1000F7EFF7F7C1F7FFF7EFEFF7E79DF7BFBD86
:100C200081BDBDEFBDFDBDBDBDBBBFBFBDBDF7BD82
:100C3000BBBFBDB9BDBFB5BBBDEFBDDBA5DBEFDF46
:100C400000000000000000000000000000000000A4
:100C50000000000000000000000000000000000094
:100C60000000000000000000000000000000000084
:100C70000000000000000000000000000000000074
:100C800000000000F0F0F0F055550000200A0000D0
:100C9000081008083E0800081010081862084042B2
:100CA0007E42421042024242424440404242084296
:100CB0004440424642404A44421042245A241020B2
:100CC0000000000000000000000000000000000024
:100CD0000000000000000000000000000000000014
:100CE0000000000000000000000000000000000004
:100CF00000000000000000000000000000000000F4
:100D0000FFFFFFFF0F0F0F0F5555FFFF81C1EFF7DB
:100D1000FBDFEFFBFFF7FFEBDFEFF7E7C3C181C3BB
:100D2000F7C3C3EFC3C3BD83C38781BFC3BDC1C303
:100D3000BD81BDBDC3BFC3BDC3EFC3E7DBBDEF8195
:100D400000000000000000000000000000000000A3
:100D50000000000000000000000000000000000093
:100D60000000000000000000000000000000000083
:100D70000000000000000000000000000000000073
:100D800000000000F0F0F0F0AAAA00007E3E10087B
:100D90000420100400080014201008183C3E7E3C7B
:100DA000083C3C103C3C427C3C787E403C423E3C13
:100DB000427E42423C403C423C103C182442107E61
:100DC0000000000000000000000000000000000023
:100DD0000000000000000000000000000000000013
:100DE0000000000000000000000000000000000003
:100DF00000000000000000000000000000000000F3
:100E0000FFFFFFFF0F0F0F0FAAAAFFFFFFF7FFFF64
:100E1000FFFFFFFFFFFFFFFFFFDFEFFFFFFFFFFF12
:100E2000FFFFFFFFFFFFFFFFFFFFFFFFFFFFFFFFD2
:100E3000FFFFFFFFFFFFFFFFFFFFFFFFFFFFFFFFC2
:100E400000000000000000000000000000000000A2
:100E50000000000000000000000000000000000092
:100E60000000000000000000000000000000000082
:100E70000000000000000000000000000000000072
:100E800000000000F0F0F0F05555000000080000F0
:100E90000000000000000000002010000000000022
:100EA0000000000000000000000000000000000042
:100EB0000000000000000000000000000000000032
:100EC0000000000000000000000000000000000022
:100ED0000000000000000000000000000000000012
:100EE0000000000000000000000000000000000002
:100EF00000000000000000000000000000000000F2
:100F0000D3FD01FF7FC3CB032A16402218401846A9
:100F1000A7C2F107C3F507FF2A16407EA7C000004D
:100F2000CD490018F7FFFFFFC39D19F1D9E3D9C9D7
:100F3000C52A1440E5C388140DC24500E105C8CB9D
:100F4000D9ED4FFBE9D1C818F82A164023221640E4
:100F50007EFE7FC018F6E16EFD7500ED7B0240CD90
:100F60000702C3BC14FF083CFA6D00280208C90838
:100F7000F5C5D5E52A0C40CBFC76D3FDDDE93F3D38
:100F8000283B2638292B2C363C2A37391D1E1F209A
:100F9000211C2524232235342E3A3E7631302F2D44
:100FA000001B3233270E190F18E3E1E4E5E2C0D944
:100FB000E0DBDD75DADEDF7277747370710B1110B0
:100FC0000DDC79141516D80C1A121317CDCEC17872
:100FD000CACBCCD1D2C7C8C9CF40787878787878D6
:100FE00078787878C2D3C4D6D578D4C6C5D0787886
:100FF00042D741080A098A8981820784060102874B
:10100000040577788503838B91908D8678929596E9
:10101000888F0B8B26B93926A78F283429AA3B261F
:10102000B1312AB3382EB32834B83926B32638B3B1
:101030002628B82639B331B32A3DB52E33B9383610
:10104000B7382CB32627B8352A2AB03A38B73839FA
:10105000378D282D378D3334B9179734B72633A9F8
:10106000139412941392392D2AB339B438392AB50E
:101070003135372E33B931312E38B9383934B538A6
:101080003134BC2B2638B9332ABC3828373431B137
:10109000283433B9292EB2372AB22B34B72C34393D
:1010A000B42C34383AA72E33353AB9313426A93125
:1010B0002E38B9312AB935263A38AA332A3DB935FE
:1010C0003430AA35372E33B9353134B9373AB338DD
:1010D000263BAA372633A92EAB2831B83A3335310F
:1010E00034B928312A26B7372A393A37B328343564
:1010F000BE3733A92E33302A3E8D35AE23EB2A146A
:101100004037ED52EBD0E1213B407E17AE17D03E89
:101110007F080611D3FE10FED3FD08173008CBFE62
:10112000F5C5D5E51803CBB6C92A34402B3E7FA4BC
:10113000B57C2003171802463767223440D0CDBB58
:1011400002ED4B254022254078C602ED423A274069
:10115000B4B558060B213B40CB862008CB7ECBC6CE
:10116000C80500372127403FCB1010FE467BFEFE0E
:101170009F061FB6A01F77D3FF2A0C40CBFCCD9251
:1011800002ED5F0101193EF5CDB5022BCD9202C3F0
:101190002902DDE1FD4E28FDCB3B7E280C79ED4494
:1011A0003C08D3FEE1D1C1F1C9D30076CD2902D3E9
:1011B00001C9E3DDE9ED4F3EDDFBE921FFFF01FE63
:1011C000FEED78F601F6E0572FFE019FB0A56F7C8B
:1011D000A267CB00ED7838ED1FCB141717179FE6E9
:1011E00018C61F322840C9FDCB3B7EC876D3FDFD13
:1011F000CB3BBEC9CF0ECDA80338F9EBEDFDC3073D
:10120000020F302E10FE1B7AB320F4CD1E03CB7ECE
:101210002328F8210940CD1E03CDFC0118F85E37C4
:10122000CB13C89FE605C6044FD3FF062310FECD9F
:10123000460F3072061E10FE0D20EEA710FD18E0BE
:10124000CDA803CB12CB0AEBEDFCC30702010600CD
:101250003E7FDBFED3FF1F30491717382810F1F10E
:10126000BAD2E503626BCD4C03CB7A792003BE2062
:10127000D6231730F1FD341521094050CD4C0371B0
:10128000CDFC0118F6D51E94061A1DDBFE17CB7B8C
:101290007B38F510F5D12004FE5630B23FCB11302B
:1012A000ADC97AA728BBCF0CCD550F3A014087FABC
:1012B0009A0DE1D0E5CDE702CDF813626B0DF80988
:1012C000CBFEC9CDE702ED4B04400B60693E3F36D3
:1012D000022BBC20FAA7ED4209233006352803353E
:1012E00028F32204402A04402B363E2BF92B2B22D4
:1012F00002403E1EED47ED56FD210040FD363B40CD
:10130000217D40220C40061936762310FB22104026
:10131000CD9A14CDAD14CD0702CD2A0A2A0A40ED8C
:101320005B2340A7ED52EB300419222340CDD809AE
:101330002801EBCD3E07FD351E20372A0A40CDD8C7
:10134000092A164037ED52212340300BEB7E23ED66
:10135000A01218C5210A405E2356E5EB23CDD8091B
:10136000CDBB05E1FDCB2D6E2008722B7318AACDE5
:10137000AD142A14407EFE7E2008010600CD600ACE
:1013800018F3FE762320EECD3705CD1F0A2A144030
:10139000FD3600FFCD6607FDCB007E20243A2240BB
:1013A000FE18301D3C322240470E01CD1809545D15
:1013B0007E2BBE20FC23EB3A0540FE4DDC5D0A1877
:1013C000C9210000221840213B40D300CB4628FC15
:1013D000D30100ED4B2540CD4B0FCDBD0730933AE7
:1013E00006403DFA0805200F3206401D7BD62738FF
:1013F000015F21CC00180E7EFE76282FFE40CBFF29
:10140000381921C70019180D7EFDCB01562007C6DB
:10141000C0FEE630017EFEF0EA2D055FCD37057B8C
:10142000CD2605C37204CD9B0912C93E785F218287
:101430000419194E2346C52A1440FDCB2D6E2016E3
:10144000FDCB01967EFE7FC823CDB40728F6FE268D
:1014500038F2FEDE28EAFDCB01D618E8010100C310
:10146000600A9F05540476057F05AF05C4050C0688
:101470008B05AF05AF05CD93057E367F2318092375
:101480007EFE762818367F2B771898CD9305CD5C95
:101490000518F62BED5B14401AFE7FC0D118EA2A1E
:1014A0000A40CDD809EBCDBB05210B40C364047BBA
:1014B000E60732064018E6EB11C2047EE6C020F7CC
:1014C00056235EC9CD1F0A216F04E5FDCB2D6EC0EA
:1014D0002A1440220E402121182239402A0A40CDE8
:1014E000D809CDBB057AB3C82BCDA50A234E234618
:1014F00023ED5B0E403E7F1213E5211D001909ED1F
:1015000072E1D0EDB0EBD1CDA6141891CD1F0A2118
:101510007204FDCB2D6E20112A14407EFEFF28069A
:10152000CDE208CD2A0A211904E5CDBA0CE1CD3768
:1015300005CD5C05CD730A201578B1C2E0060B0B12
:10154000ED430740FD362202ED5B0C401813FE769A
:101550002812ED4B3040CD1809ED5B2940FD3622B5
:1015600002DFFE76CA1304FD360180EB222940EB30
:10157000CD4D00CDC10CFDCB018E3EC0FD7719CD08
:10158000A314FDCB2DAEFDCB007E28222A2940A638
:10159000201C56235EED530740235E235623EB1990
:1015A000CD460F38C7210040CB7E2802360CFDCB3C
:1015B000387ECC7108012101CD18093A0040ED4B6D
:1015C00007403C280CFE09200103ED432B4020017D
:1015D0000BCDEB073E18D7CD980ACDAD14C3C1048F
:1015E000ED430A402A1640EB211304E52A1A40ED88
:1015F00052E5C5CDE702CD2A0AE1CDD8092006CDB6
:10160000F209CD600AC1793DB0C8C5030303032BBD
:10161000CD9E09CD0702C1C5132A1A402BEDB82A69
:101620000A40EBC1702B712B732B72C9FDCB01CE1D
:10163000CDA70E78E63F6769220A40CDD8091E0083
:10164000CD450718FBED4B0A40CDEA091692280557
:10165000110000CB13FD731E7EFE40C1D0C5CDA589
:101660000A237AD72323221640FDCB01C6ED4B185F
:10167000402A1640A7ED4220033EB8D72A16407EE6
:1016800023CDB40722164028E4FE7F2810FE7628DA
:101690005DCB772805CD4B0918D3D718D03A064033
:1016A00006ABA720053A014006B01F1FE60180CD1A
:1016B000F50718B9FE7EC02323232323C91600CBC8
:1016C000289FF6262E05958537CB1938FA0CC04889
:1016D0002D2E0120F2217D005F1937C97BA7F81854
:1016E00010AF093C38FCED423D28F11E1C83A728B1
:1016F00004FDCB0186D9E5FDCB014E2005CD0808C0
:101700001803CD5108E1D9C957ED4B394079FE2175
:10171000281A3E76BA28302A0E40BE7A20200D20A4
:101720001923220E400E2105ED43394078FDBE22DB
:101730002803A720DD2E04C35800CD9B09EB772397
:10174000220E40FD3539C90E2105FDCB01C6C31857
:1017500009FE76281C4F3A3840E67FFE5C6F264033
:10176000CC7108712CFD7538C916162A0C40231847
:10177000051601213C40CDE702C5E5AF5FD3FBE193
:10178000CD460F38051FD3FBCF0CDBFB87FADE08F5
:1017900030EEE5D57AFE029FA307A3574E7923FECC
:1017A000762824E5CB278787260FCB14836FCB11B0
:1017B0009FAE4F06087ACB011F67DBFB1F30FB7C17
:1017C000D3FB10F1E118D5DBFB1F30FB7A0FD3FB05
:1017D000D11CCB5B28A7C11520A03E04D3FBCD07AD
:1017E00002C1215C40367606202B360010FB7DCBF3
:1017F000FF323840C93E1790380BFDBE22DA35085B
:101800003C473E1F91DAAD0EC6024FFDCB014E287C
:10181000073E5D91323840C9ED4339402A104051AE
:101820003E22914F3E76042BBE20FC10FA23EDB1F0
:101830002B220E4037E015C8C5CD9E09C141626B11
:1018400036002B10FBEB23220E40C9F5CD75093075
:1018500008FDCB01462002AFD70AE63FD70A03872F
:1018600030F7C1CB78C8FE1A2803FE38D8AFFDCBBD
:1018700001C6C3F507E5211101CB7F2802E63FFE33
:101880004330104704CB7E2328FB10F9CB7720028E
:10189000FE183F444DE1D00AC6E4C9010100E5CD80
:1018A000C50EE1CDAD092A1C40EBEDB8C9F5E52127
:1018B0000C403E095E2356E3A7ED5219E33009D5EB
:1018C000EB09EB722B7323D1233D20E8EBD1F1A779
:1018D000ED52444D0319EBC9E5217D40545DC1CD66
:1018E000EA09D0C5CDF209EB18F47EB8C0237E2BEF
:1018F000B9C9E57EFE403817CB6F281487FA010A74
:101900003F01050030020E1117237E30FB1806231D
:10191000234E23462309D1A7ED52444D19EBC9FDAF
:101920004622C5CD2C0AC10518020618FDCB018E32
:101930000E21C5CD1809C13A0540FE4D3814FDCB26
:101940003AFEAFCDF5072A39407DB4E67E20F3C3D9
:101950001809545D2B480600EDB02A1040CD170A37
:10196000C5782F47792F4F03CDAD09EBE119D5EDA0
:10197000B0E1C92A1440CD4D00DFFDCB2D6EC02152
:101980005D40221C40CD4815CD8A15380421F0D881
:1019900009DA9A0DBFC3BC14D5E5AFCB782020601F
:1019A000691EFF1808D556235EE5EB1E000118FCE2
:1019B000CDE107019CFFCDE1070EF6CDE1077DCD1E
:1019C000EB07E1D1C9CDA60DE1C8E9FDCB01CE7E83
:1019D000FE76CA840BD61ACE002869FEA7201BE724
:1019E000CD920DFE1AC29A0DE7CD920DCD4E0BEFA2
:1019F0000134CDF50BCDF508183DFEA82033E7CD19
:101A0000920DCD4E0BCD020CC2AD0EE61F4FFDCB9D
:101A1000014E280AFD9638CBFFC63CD47108FD86DE
:101A200039FE213A3A40DE01CDFA08FDCB01C61855
:101A300006CD550FCD550BDFD61ACE002806CD1D8D
:101A40000DC3840BD48B0BE7FE76C8C3D50ACDA695
:101A50000DC0E118E2CDC50AFDCB0176CCF8132804
:101A60000AC3DB153E0BD7ED5B184078B10BC81AE3
:101A700013ED531840CB7728EDFEC028E7C5CD4BBA
:101A800009C118E3CDC50A3E76D7C9CDC50AFDCB3D
:101A900001C6AFD7ED4B394079FDCB014E28053E4D
:101AA0005DFD96380E11B930020E01CD0B09C9CD7E
:101AB000F50BED4336403E2B90DAAD0E473E01CBA1
:101AC0002830023E04CB29300107F5CDF5087E070A
:101AD000FE1030060F3002EE8F47119E0C3A304058
:101AE00093FAE90BF12FA01802F1B0FE083802EECC
:101AF0008FD9D7D9C9CD020C47C5CD020C59C151D8
:101B00004FC9CDCD15DAAD0E0E01C80EFFC9FD4689
:101B1000220E21CD1809CD9B097E12FD343A2A0CE4
:101B20004023545DEDB1C35D0A8B8D2D7F814975D6
:101B30005F40422B171F3752450F6D2B442D5A3BE8
:101B40004C450D525A4D156A0114020600810E06CD
:101B5000DE05AB0D0600B50E00DC0C00D80E04143B
:101B600006DF0605B90D04002E0E05CF0A0100E9B7
:101B70000E050914056A0D00C30303AF0E033007F9
:101B8000061A0600920E036C0E05400305F60200CD
:101B90007C0E009A14002A0A061A0600AF0B061AD9
:101BA0000600AF0B000E0C0600320F002B0F0023B7
:101BB0000F00690805CB0A032C07FD360101CD7320
:101BC0000ACDBC1421004036FF212D40CB6E280EDB
:101BD000FEE37EC26F0DCDA60DC8CF0CCF08DF0689
:101BE00000FE76C84FE779D6E1383B4F21290C0932
:101BF0004E0918032A30407E2322304001F40CC5E0
:101C00004FFE0B300B21160D0600094E09E5DFC90A
:101C1000DFB92012E7C91725530F6B1376CDA60D38
:101C2000C0C17EFE76C81872FE76CD9C0DBFC1CCB9
:101C30001D0DEB2A30404E2346EBC5C9CD1C11FDCE
:101C4000362D003008FDCB2DCE2018CF01CCA711AA
:101C5000FDCB0176200DAFCDA60DC4F813212D408C
:101C6000B677EBED432E40221240C9C13A0140F550
:101C7000CD550FF1012113FD5601AAE640201BCBE3
:101C80007A20B7189DCD1C11F579F69F3C200BF1F9
:101C900018ADCD550FFDCB0176C0CF0B20F4CDA6EE
:101CA0000DC8EFA034C9FDCB017EC9CDA60D280615
:101CB000EF02341AA7C8C3DE0CFEE02009E7CD927C
:101CC0000DCD1D0D1806CD1D0DEFA134EFC0020185
:101CD000E00134CD2113221F402B7ECBFE010600F4
:101CE00009073806CB21CD9E0923E5EF020234E136
:101CF000EB0E0AEDB02A0740EB13732372CD5A0E98
:101D0000D0FDCB087EC0FD462ECBB02A29407EE612
:101D1000C02017C5CDF209C1232323CD4C00DFFE1F
:101D2000F3EB20EAEBE7EBB820E4222940C9FDCB36
:101D30002D4EC24B0D2A1240CB7E281C23221F4061
:101D4000EFE0E20FC00234CD5A0ED82A1F40110F27
:101D500000195E2356EB182ECF00EFE1E0E23200CF
:101D600002010333000434A7C93437C9CDA70E7864
:101D7000B12004ED4B3440ED433240C92A2B4018CA
:101D800005CDA70E60697CFEF03022CDD80922294E
:101D900040C9CDCD1538162802ED44F5CDA70EF17A
:101DA000FDCB007EC802C9CD8A153801C8CF0ACD47
:101DB000810EC39A142A074023E3E5ED730240CD58
:101DC000810E0106002A1C40093808EB2124001965
:101DD000ED72D82E03C35800E1E37CFE3E2806EDE9
:101DE00073024018A1E3E5CF06FDCB087E2032CD7B
:101DF000A314212D40CBEECBB63A0140E6400102C0
:101E00000020020E04B677F73676790F0F38053EBC
:101E10000B122B772B367F2A3940223040E1C372D8
:101E200004CF07CDE702FDCB3BB6C9FDCB3BF6C3E4
:101E30000702CDA70ECDE7026069CD2D02FD363534
:101E4000FFCD070218053E7FDBFE1FFDCB3B863E24
:101E5000FF322740C9DF0600C5FE40202FCDA60D6A
:101E60002828ED4B3240CD2015EFA10F3037160456
:101E70003080410000802E02A1032D34CD8A15ED63
:101E80004332407EA72803D61077180DFE42200D5E
:101E9000CDA60D2804EFA33434E7C38310FE412000
:101EA00011CDBB02444D5114C4BD077A8A424FEB99
:101EB000183BCDD214386EFE1BCA471001D809FE5C
:101EC00016285DFE10200FCD4900CD550FFE1120C4
:101ED0002ECD49001822FE0B2028CD4900E518031D
:101EE000CD4900FE0B2014D1A7ED52444D210140F5
:101EF000CBB6CB7EC4C312E7C38810FE7620E1C305
:101F00009A0DD6C438F901EC04FE13281330F006FC
:101F100010C6D94FFEDC3002CBB1FEEA3802CBB995
:101F2000C5E7C3590FFE26381ECD1C11DA4B0DCC68
:101F3000A7113A0140FEC0384E23ED5B1C40CDF6A0
:101F400019EB221C401840CDA60D2023CDD914DF5B
:101F5000010600CD9E0923367E23EB2A1C400E0588
:101F6000A7ED42221C40EDB0EB2BCD4C001814E73E
:101F7000FE7E20FB23ED5B1C40CDF619ED531C408B
:101F8000221640FDCB01F6DFFE10200CFDCB0176C2
:101F9000202ACD6312E718F001C300FE12381DD6C7
:101FA000163004C60D180EFE03380AD6C2380DFED0
:101FB000063009C603814F214C100946D17AB83842
:101FC0002CA7CA1800C5D5CDA60D28097BE63F472A
:101FD000EF373418097BFDAE01E640C29A0DD121DE
:101FE0000140CBF6CB7B2002CBB6C118CFD579FD13
:101FF000CB01762015E63FC6084FFE102004CBF13A
:10200000180838D7FE172802CBF9C5E7C3590F06C1
:1020100008080A020305050505050506FDCB01F6BE
:10202000DFCDCE14D29A0DE54FE7E5CBA9FE1028FF
:1020300017CBF1FE0D280CCBE9CDD214300ACBB171
:10204000E718F6E7FDCB01B641CDA60D200879E6ED
:10205000E0CBFF4F18342A10407EE67F282AB920B3
:102060001F1787F29511382DD1D5E5231A13A7280C
:10207000FBBE28F7F680BE20061ACDD2143015E13B
:10208000C5CDF209EBC118D1CBF8D1DFFE1028097C
:10209000CBE8180DD1D1D1E5DFCDD2143003E7184C
:1020A000F8E1CB10CB70C9AF47CB79204BCB7E206A
:1020B0000E3C234E234623EBCDC312DFC35A12231B
:1020C000232346CB71280A0528E8EBDFFE102061A8
:1020D000EBEB1824E5DFE1FE1A2820CB792852CB60
:1020E000712006FE11203CE7C9FE11286CFEDF209E
:1020F00032DF2B221640185E210000E5E7E179FE71
:10210000C02009DFFE112851FEDF28E5C5E5CDFF1F
:1021100012E3EBCDDD1238190BCD051309D1C11037
:10212000B3CB792066E5CB712013424BDFFE11283B
:1021300002CF02E7E1110500CD051309C9CDFF1259
:10214000E3CD0513C10923424BEBCDC212DFFE11D3
:102150002807FE1A20DBCD6312E7FE1028F8FDCB1E
:1021600001B6C9CDA60DC4F813E7FE112850D5AFAE
:10217000F5C5110100DFE1FEDF2817F1CDDE12F514
:102180005059E5DFE1FEDF2809FE11C29A0D626BAE
:102190001813E5E7E1FE11280CF1CDDE12F5DF6042
:1021A00069FE1120E6F1E3192BE3A7ED52010000CF
:1021B000380723A7FA3112444DD1FDCB01B6CDA685
:1021C0000DC8AFC5CDEB19C12A1C4077237323720C
:1021D0002371237023221C40FDCB01B6C9AFD5E586
:1021E000F5CD920DF1CDA60D2812F5CDA70ED17823
:1021F000B1372805E1E5A7ED427ADE00E1D1C9EB70
:10220000235E2356C9CDA60DC8C506107C4D2100FE
:1022100000293806CB1117300419DAD30E10F2C199
:10222000C92A1240FDCB2D4E284401050003237E10
:10223000A728FBCDD21438F5FE0DCAC813F7D52A4E
:1022400012401B79D606473E40280E237EA728FB66
:10225000131210F7F680123E802A1240AEE1CDE74D
:1022600013E5EF0234E1010500A7ED421840FDCB74
:10227000017628061106001918E72A1240ED4B2EA8
:1022800040FDCB2D46203078B1C8E5F7D5C5545D6B
:10229000233600EDB8E5CDF813E1E3A7ED420930B0
:1022A00002444DE3EB78B12802EDB0C1D1E1EB7807
:1022B000B1C8D5EDB0E1C92B2B2B7EE5C5CDCE1332
:1022C000C1E1030303C3600A3E602A1240AEF5CDAC
:1022D000F813EB09E5030303F7EBE10B0BC5EDB8CE
:1022E000EBC10B702B71F1F5CDC714F12B772A1AC6
:1022F000402214402B3680C92A1C402B462B4E2BE3
:10230000562B5E2B7E221C40C9CD1C11C29A0DCDCE
:10231000A60D2008CBB1CDA711CD1D0D3808C5CD18
:10232000F209CD600AC1CBF90600C5210100CB71CD
:1023300020022E05EBE72640CDDD12DA3112E1C591
:1023400024E56069CD0513EBDFFE1A28E8FE1120B5
:10235000BBE7C17968260023232919DAD30ED5C536
:10236000E5444D2A14402BCD9E092377C10B0B0B5E
:1023700023712370F12377626B1B3600C1EDB8C166
:10238000702B712B3D20F8C92A1A402BCD9E0923B2
:1023900023C1ED431440C1EB23C92A1040368023EA
:1023A0002214402A1440221A40221C40C92A1440F8
:1023B000367F23367623FD36220218EA215D40223D
:1023C0001F402A1A4018E2ED5B1440C35D0AFE2646
:1023D0001802FE1C3FD0FE40C9CD4815FE1B20153B
:1023E000EFA1C00234E7CD1415380AEFE0A405C010
:1023F000040F3418F0FE2AC0FD365DFFE7FE1528F5
:1024000007FE162004FD345DE7CD4815EFE000021D
:10241000183834C9FE1CD8FE263FD8D61C4F0600FB
:10242000FD210040C5EFA034C1369178A720077781
:10243000B1C8414E368935CB21CB1030F9CB38CBE2
:1024400019237023712B2BC9F5EFA034F1CD14158E
:10245000D8EF01A4040F34E718F3EF2D32C00227A0
:10246000A1032D3200222D303340032D32000C0108
:1024700002013080481896802F040201A4E0000475
:10248000042F0205012FDA0234C9CDF813A7200565
:10249000474FF5183143594AD6913FCB78F5CBF8E1
:1024A00038243CED44FE08380659480600D608A7F3
:1024B000577B072807CB38CB191520F9300803784C
:1024C000B12003F137F5C5EF34C1F179C9CD8A15D3
:1024D000D8F505042803F137C9F1C9EF2D32000BF7
:1024E0002D33000D02343E1CD7C927343E16D7EFDA
:1024F000347ECD1D15EF307800800330EF1A209A1E
:10250000850424C1303400031838A20F2434216B11
:10251000403690060A23E5C5EFA42E0134CDCD1533
:10252000F690C1E17710EE23010800E52B7EFE90C6
:1025300028FAED42E57EC66BF5F1237ECE0027F545
:10254000E60F77CBFE28F2F1E1060636802B10FB72
:10255000EF02E134CDCD152802ED445F1C1CE12BC8
:102560001D7EE60F28F97BD605FE08F28216FEF6E0
:10257000FA8216C6062848FAB21647CDD01610FBC6
:10258000184043CDD016CDC2163E2AD778A7F29870
:1025900016ED44473E1618023E15D77806FF04D6BE
:1025A0000A30FBC60A4F78A72803CDEB0779CDEB9D
:1025B00007C9ED44473E1BD73E1CD710FD18093E06
:1025C0001CD73534E83E1BD73534E8CDD01618F883
:1025D0007EE60FCDEB072BC97E3600A7C823CB7E46
:1025E000CBFE2BC8C501050009414F372B7E2FCEEE
:1025F000007710F879C1C9E5F54E23467723794E67
:10260000C5234E2346EB575ED52356235ED5D9D13D
:10261000E1C1D92356235EF1E1C9A7C8FE213016D6
:10262000C547D9CB2DCB1ACB1BD9CB1ACB1B10F25C
:10263000C1D0CD4117C0D9AF2E00575DD9110000D0
:10264000C91CC014C0D91C200114D9C91AA7C813A9
:102650001AEE80121BD9E5D9D5E5CDD81647EBCDBA
:10266000D8164FB830037841EBF590CDF716CD1A58
:1026700017F1E177E5686119D9EBED4AEB7C8D6FD5
:102680001FADD9EBE11F30083E01CD1A17342823C6
:10269000D97DE680D923772B281F7BED443F5F7AD5
:1026A0002FCE0057D97B2FCE005F7A2FCE00300778
:1026B0001FD934CA8018D957D9AF186C373534C8E8
:1026C00023AECBFE2BC9AFCDBC17D8D9E5D9D5EBFE
:1026D000CDBC17EB385AE5CDF71678A7ED62D9E5F2
:1026E000ED62D906211811300519D9ED5AD9D9CB87
:1026F0001CCB1DD9CB1CCB1DD9CB18CB19D9CB19D1
:102700001F10E4EBD9EBD9C1E178812001A73D3F4F
:10271000173F1FF219183068A73C20083806D9CB9C
:102720007AD9205C77D978D930157EA73E802801E8
:10273000AFD9A2CD38170777382E23772B18290663
:1027400020D9CB7AD9201207CB13CB12D9CB13CBFC
:1027500012D93528D710EA18D717300CCD411720D9
:1027600007D91680D9342818E523D9D5D9C17817C7
:10277000CB161F77237123722373E1D1D9E1D9C915
:10278000CF05EBAFCDBC1738F7EBCDBC17D8D9E5EB
:10279000D9D5E5CDF716D9E56069D96168AF06DF0F
:1027A000181017CB11D9CB11CB10D929D9ED6AD973
:1027B0003810ED52D9ED52D9300F19D9ED5AD9A7A9
:1027C0001808A7ED52D9ED52D93704FAA218F52806
:1027D000E15F51D95950F1CB18F1CB18D9C1E1784B
:1027E00091C310187EFE81300636003E201805D6B3
:1027F000A0F0ED44D5EB2B47CB38CB38CB382805B0
:1028000036002B10FBE6072809473EFFCB2710FCBC
:10281000A677EBD1C900B00031003000F1490FDAE2
:10282000A234202F1C721AE3194C17C6178218E223
:102830001DED1AF31A031B031B031B031B031B03CE
:102840001B5517F81A031B031B031B031B031B0356
:102850001B621BA01A061CA41B111C491D3E1D6EE9
:102860001DC41DD41D761DA91C5B1C461CDB1DAFA1
:102870001AAA1ABE1AC51AD51B8F1BD51AF61937F4
:102880001C231CFC19171CDB1ACE1A2B00181DE484
:1028900018E4195A157F1A511A631A451ACD851B67
:1028A00078321E40D9E3D9ED531C40D97E23E5A7E9
:1028B000F2C21957E6600F0F0F0FC6726F7AE61F4C
:1028C000180EFE183008D901FBFF545D09D9076FB7
:1028D0001123192600195E235621A719E3D5D9ED36
:1028E0004B1D40C9F13A1E40D918C3D5E50105007A
:1028F000CDC50EE1D1C9CDEB19EDB0C9626BCDEB01
:1029000019D9E5D9E3C57EE6C007074F0C7EE63F3F
:102910002002237EC650123E059123130600EDB01F
:10292000C1E3D9E1D947AF05C8121318FAA7C8F512
:10293000D5110000CDFE19D1F13D18F24F070781E6
:102940004F060009C9D52A1F40CD3C1ACDF619E122
:10295000C9626BD9E5211519D9CD2D1ACDFE19D92A
:10296000E1D9C9E5EB2A1F40CD3C1AEBCDF619EBB6
:10297000E1C906051A4EEB1271231310F7EBC94794
:10298000CDA0192D0FC002A0C22DE004E2C1033476
:10299000CDFC19CDA4190F01C20231EEE10334C9F7
:1029A0007EA7C8237EEE80772BC923CBBE2BC923FD
:1029B0007E2B353437C4E01A2307CB1E2BC9CDA795
:1029C0000E0AC31D15CDA70E212015E5C5C97EA78A
:1029D000C83EFF18077EED443F1805AF23AE2B0716
:1029E000E5060536002310FBE1D03681C91AA7C8D9
:1029F0003718ED1AA7C018E81AA7C0D51BAF121BCD
:102A000012D1C978D608CB5720013D0F3008F5E523
:102A1000CD721AD1EBF1CB5720070FF5CD4C17181B
:102A2000330FF5CDF813D5C5CDF813E17CB5E378B8
:102A3000200BB1C12804F13F1816F11813B1280D6D
:102A40001A96380920ED0B1323E32B18DFC1F1A7E9
:102A5000F5EFA034F1F5DCD51ACDCE1AF10FD4D5AF
:102A60001AC9CDF813D5C5CDF813E1E5D5C509448C
:102A70004DF7CDC312C1E178B12802EDB0C1E178C4
:102A8000B12802EDB02A1C4011FBFFE519D1C9CDD8
:102A9000CD15380E200CF5010100F7F112CDC3124F
:102AA000EBC9CF0A2A1640E5CDF813D503F7E1EDBF
:102AB000531640D5EDB0EB2B3676FDCB01BECD9253
:102AC0000DCD220DE1221640FDCB01FECD550FE1CB
:102AD00022164018B0010100F736762A3940E52E5B
:102AE000FF2239402A0E40E5ED530E40D5CDDB15CF
:102AF000D12A0E40A7ED52444DE1220E40E1223989
:102B000040CDC312EBC9CDF81378B128011AC31D0B
:102B100015CDF813C32015D9E5211E4035E1200459
:102B200023D9C9D95EAFCB7B28012F5719D9C91A30
:102B3000A720F0D923D9C9EFC0022DE00524E00178
:102B4000C00403E034C9EF2D3200043634C92D36F9
:102B5000C003E0012C0003A10334C9EF30F138AA0F
:102B60003B29042D24C3032D0FA103881336586578
:102B7000669D786540A26032C9E721F7AF24EB2F4C
:102B8000B0B014EE7EBB9458F13A7EF8CFE334CD6A
:102B9000CD1520073803863009CF05380796300455
:102BA000ED4477C9EF02A034C9EF2D33000434CFD0
:102BB00009A002347E3680CD1D15EF3038000301A8
:102BC0002D30F04CCCCCCD0333000801A1030134EF
:102BD00034EF0130F0317217F80401A203A2032D83
:102BE00030322004A2038C11AC140956DAA55930F6
:102BF000C55C90AA9E706F61A1CBDA96A4319FB498
:102C0000E7A0FE5CFCEA1B43CA36EDA79C7E5EF0A3
:102C10006E238093040F34C9EF30EE22F9836E04E3
:102C20002DA20F24032D0F2D0F2D27A1032D33C00F
:102C300000040234C9A103013200021834C9EF357F
:102C400027A103E00006182F03EF352D2D042D0FCB
:102C5000A1038614E65C1F0BA38F38EEE91563BB56
:102C600023EE920DCDEDF1235D1BEA0434C9EF2D67
:102C70001C011D0534C97EFE81380EEFA118010527
:102C80002D32A3010006182F03EFA0012D2D042DD6
:102C90000FA1038C10B2130E55E48D5839BC5B980C
:102CA000FD9E003675A0DBE8B46342C4E6B5093684
:102CB000BEE936731B5DECD8DE63BEF061A1B30CD8
:102CC000040F34C9EF2D2D04A1031825A10F0521F0
:102CD0002D0F34C9EF1FA3031834C9EF2D2C001E8C
:102CE000A234EF012D2C0007220434C35B1C022DFB
:102CF0002C0009A001330006A1010502A134C9FF7F
:102D00000000000000000000F0F0F0F00000000003
:102D10000F0F0F0F00000000FFFFFFFF000000007B
:102D200000000000F0F0F0F0F0F0F0F0F0F0F0F063
:102D30000F0F0F0FF0F0F0F0FFFFFFFFF0F0F0F0DB
:102D4000AA55AA55AA55AA5500000000AA55AA5589
:102D5000AA55AA550000000000242400000000002D
:102D6000001C227820207E0000083E283E0A3E08F3
:102D70000000001000001000003C420408000800A1
:102D8000000408080808040000201010101020009B
:102D900000001008040810000000040810080400D7
:102DA0000000003E003E0000000008083E08080049
:102DB000000000003E000000000014083E0814005F
:102DC0000000020408102000000010000010102075
:102DD00000000000000808100000000000181800A3
:102DE000003C464A52623C000018280808083E0091
:102DF000003C42023C407E00003C420C02423C004F
:102E000000081828487E0800007E407C02423C00F2
:102E1000003C407C42423C00007E0204081010004E
:102E2000003C423C42423C00003C42423E023C00EC
:102E3000003C42427E424200007C427C42427C0096
:102E4000003C424040423C0000784442424478000A
:102E5000007E407C40407E00007E407C4040400040
:102E6000003C42404E423C000042427E4242420010
:102E7000003E080808083E000002020242423C00F0
:102E800000444870484442000040404040407E00BA
:102E90000042665A42424200004262524A464200A2
:102EA000003C424242423C00007C42427C404000A6
:102EB000003C4242524A3C00007C42427C44420078
:102EC000003C403C02423C0000FE1010101010007C
:102ED0000042424242423C00004242424224180028
:102EE00000424242425A2400004224181824420060
:102EF0000082442810101000007E040810207E007C
:102F000011241FBECFEFD0E1DEBFCDBF11E0A0E0A6
:102F1000B1E0EAE4F0E702C005900D92A230B107FB
:102F2000D9F720E1A2E0B1E001C01D92AC32B207B6
:102F3000E1F70E94F5370C9423380C94000090912F
:102F4000060190FD30C0803F21F49160909306010E
:102F500008958093020187FD25C0863659F480913B
:102F60001F018E7F80931F01809123018E7F8093AC
:102F700023010895E82FF0E0E059FF4FE491EF3F7F
:102F800089F0AE2FA295AF70B0E0A15EBE4FE770A2
:102F900081E090E001C0880FEA95EAF780959C9166
:102FA00089238C9308959E7F9093060110920201CD
:102FB00087FDF8CF863649F480911F0181608093A8
:102FC0001F01809123018160D2CFE82FF0E0E0590A
:102FD000FF4FE491EF3F31F3AE2FA295AF70B0E019
:102FE000A15EBE4FE77021E030E001C0220FEA95FC
:102FF000EAF78C91822BD5CF8091C00087FF04C067
:103000008091C6000E949F170895109206011092A9
:10301000C00080E18093C10086E78093C200509891
:103020002098589A289A0895689432F80895C20111
:1030300092012F5F3F4F29010E94FC330895CF93E7
:103040000E941718C82F0E941718982F8C2FCF9105
:103050000895682FC30101973C010E941A34089516
:10306000C30193012F5F3F4F39010E94E63308955A
:10307000CF93C82F692FC30101973C010E941A34D6
:10308000C30101973C016C2F0E941A34CF9108951F
:10309000CF930E943018C82F0E943018982F8C2F81
:1030A000CF910895512C412C66246A94762C2224C9
:1030B0002A9433243A941092170110921601109218
:1030C0000E01109215010895222D822D90E02F708F
:1030D000A22E332D532D507131FE23C041E030FC20
:1030E00004C08A3991050CF440E0511113C02A3014
:1030F00098F4442311F080569140282EFC01FF27BC
:10310000E051FF4F3491E32DEB73E32B90FD20C092
:103110003E2E0895263010F03F7E332E06979927D5
:10312000E8CF51110DC02A3068F430FC06C09C0174
:10313000207F31702139310504F3805A9F4FDDCF54
:103140002A3020F03061332E0696EFCF3F7EFBCF42
:10315000E160DECFCF93C1E0C80FEC2FF0E0E0518B
:10316000FF4F2491E32DEB73E22BE97E982F9F70A4
:103170009F3041F03E2E8F3711F40E9414188C2F8F
:10318000CF910895E061F6CFCF93CFEFC80FEC2F2A
:10319000F0E0E051FF4F2491E32DEB73E22BEB7E47
:1031A000982F9F7049F0E2603E2E803811F40E9403
:1031B00014188C2FCF910895E261F6CFCF93282F6A
:1031C000260F3327331FA901982F96272927C82FA9
:1031D000C60FEC2FF0E0E051FF4F8491E32DEB732D
:1031E000E82BE87E50FD0FC03E2E24FF02C06894FD
:1031F00034F8C90196958795282727FD0E94141851
:103200008C2FCF910895E160EFCFCF93DF93932D73
:10321000232D2170C22F20E0D22FC60FD11DC80F41
:10322000D11D86279E012827FE01FF27E051FF4F71
:10323000E4919B739E2B987ED0FD10C0392E24FF05
:1032400002C0689434F8C90196958795282727FD10
:103250000E9414188C2FDF91CF9108959160EECFCA
:10326000CF92DF92EF92FF929B01AC01462753274A
:1032700070E060E06901F12CE12CC80ED91EE11C60
:10328000F11C4C255D256E257F25452F562F672F78
:103290007727E32DEC7EDA01A071BB27AB2B71F40D
:1032A0003E2E44275170452B11F0689430F8820F60
:1032B000931FFF90EF90DF90CF900895E061F0CFE3
:1032C000CF92DF92EF92FF92AC01232D332D31701C
:1032D000CB01B0E0A0E0830F911DA11DB11D840FB3
:1032E000951FA11DB11D4627572770E060E04827B4
:1032F00059276A277B27C52ED62EE72EFF24287252
:10330000D0FC1EC0322EC4FE02C0689434F8009770
:1033100011F4689436F897FF02C0689437F829E0F2
:1033200076956795579547952A95D1F74C2547FF90
:1033300002C0689432F8FF90EF90DF90CF9008952C
:103340002160E0CFCF93282F261B330BA901982FA4
:1033500096272927C82FC61BEC2FF0E0E051FF4F1E
:103360008491E32DEB73E82BEA7E50FD10C0E26000
:103370003E2E24FF02C0689434F8C90196958795C3
:10338000282727FD0E9414188C2FCF910895E36001
:10339000EFCFCF93DF93932D282F261B330BE9011B
:1033A000232D217030E0C21BD30B86279E012827D6
:1033B000FE01FF27E051FF4FE4919B739E2B9A7E05
:1033C000D0FD11C09260392E24FF02C0689434F8F9
:1033D000C90196958795282727FD0E9414188C2FE0
:1033E000DF91CF9108959360EECFCF92DF92EF926D
:1033F000FF92AC01232DB0E0A0E0861B970BA10942
:10340000B109332D3170831B9109A109B1094627F8
:10341000572770E060E0482759276A277B27C52E89
:10342000D62EE72EFF242A72D0FC1FC02260322E37
:10343000C4FE02C0689434F8009711F4689436F81A
:1034400097FF02C0689437F829E0769567955795FD
:1034500047952A95D1F74C2547FF02C0689432F86A
:10346000FF90EF90DF90CF9008952360E0CFCF934F
:10347000DF930E941718C82FD82FD770D1506091B2
:103480001901D73078F4ED2FF0E0E75BF54E0C949E
:103490001D38501A7E1A811A841A871A8A1A921AAB
:1034A00060911801C695C695C695C150CF3108F0F8
:1034B0003BC0EC2FF0E0E15AF54E0C941D38B81AE1
:1034C000CC1AE41AF11AFB1A071B111B1A1B221B38
:1034D000281B2D1B321B371B3C1B411B461B481B4B
:1034E0004A1B4C1B4E1B501B521B541B561B581B7C
:1034F0005A1B5C1B5E1B601B621B641B60911B01E3
:10350000D1CF60911A01CECF60911001CBCF6091E5
:103510000F01C8CF80910F01909110010E94E633F6
:10352000682FC0CF622DBECF832D8C7E67FD1EC05D
:10353000382E932D832D8170660F682BE62FF0E0D7
:10354000E051FF4FE4919B739E2B392ED73008F04A
:10355000BDC0ED2FF0E0E155F54E0C941D386B1B0E
:103560006E1B711B741B771B7A1B811B8160E0CF64
:10357000832D8C7E60FD0EC0382E6695832D30FC29
:103580006068E62FF0E0E051FF4FE4918B738E2BE3
:10359000382EDCCF8160F0CF932D232D2D7E322E5F
:1035A000862F880F392F3170832B67FF17C021605A
:1035B000322E932DE82FF0E0E051FF4FE4919B7302
:1035C0009E2B392E682FC2CF932D232D2D7E322E88
:1035D000862F869590FD806860FDE9CF9C7E392E10
:1035E000E8CF832D8C7E67FD04C0382E660F832DB7
:1035F000C8CF8160FACF832D8C7E60FD06C0382E47
:10360000862F80786695682BF2CF8160F8CF832D66
:103610008C7E67FD04C0382E660F6160E8CF816044
:10362000FACF832D8C7E60FD03C0382E6695DFCFE8
:103630008160FBCF832D8D7B60FF08C0382E68949E
:1036400034F884CF832D8D7B61FDF8CF8064F6CF75
:10365000832D8D7B62FFFACFF1CF832D8D7B63FFAE
:10366000F5CFECCF832D8D7B64FFF0CFE7CF832D9B
:103670008D7B65FFEBCFE2CF832D8D7B66FFE6CFA1
:10368000DDCF832D8D7B67FFE1CFD8CF6E7F5ECFFF
:103690006D7F5CCF6B7F5ACF677F58CF6F7E56CFE1
:1036A0006F7D54CF6F7B52CF6F7750CF61604ECF1D
:1036B00062604CCF64604ACF686048CF606146CF9B
:1036C000606244CF606442CF606840CF609319016C
:1036D000DF91CF91089560931801FACF60931B0199
:1036E000F7CF60931A01F4CF60931001F1CF60938C
:1036F0000F01EECF80910F01909110010E941A34BA
:10370000E7CF262EE5CFFF92CF930E941718A82E61
:10371000823609F447C208F086C08F3409F4FFC12D
:10372000B8F5863409F4D4C1B8F4823409F4A9C1D7
:1037300048F4803409F48BC1813409F49AC10E94A1
:103740003C34C0C1843409F4B3C108F4A3C18091EE
:10375000150180930E0118C0893409F4BFC168F4C3
:10376000873409F4B8C1883451F78091180190E08A
:103770000E9428348093180171C18B3409F4C1C1AF
:1037800008F4B0C18D34D9F60E9448182C019AC1B2
:10379000883509F4E9C100F5823509F4CBC150F44C
:1037A000803509F4BFC1813551F6809118016091CF
:1037B0001B0163C1863509F4C2C108F0C4C1833559
:1037C00009F0BDCF0E941F184C0160911A010E94A0
:1037D0001A3460911B0167C18E3509F4D7C1B0F46A
:1037E0008A3509F4CEC108F4C7C18B3509F0A7CFDB
:1037F0000E941F184C010E94E63380931A01C401F5
:1038000001960E94E63380931B015CC1803609F467
:10381000C1C1E0911301813608F497C1809118016C
:10382000609110012AC1833A09F475C208F072C090
:10383000833709F403C208F5893609F4DFC170F44F
:10384000873609F4B7C1883609F079CF809118011D
:1038500090E00E94283480930F0100C18F3609F454
:10386000D2C1823709F4E8C18A3609F068CF809165
:103870000F0190911001BC013DC18B3709F4ECC1DF
:1038800078F4893709F4E2C108F0E4C1883709F017
:1038900056CF8091180190E00E942834282EDEC077
:1038A000813A09F4E6C108F010C2803A09F047CF26
:1038B00080910F01909110010E94E633A82E682F8D
:1038C00080911A0190911B010E941A3480910F017E
:1038D0009091100101969093100180930F018091B7
:1038E0001A0190911B01019690931B0180931A017C
:1038F000809118019091190101979093190180937B
:103900001801892B09F032C2E89432F8832D8D7E9C
:10391000382ED8C0823B09F494C208F043C08A3ADA
:1039200009F427C248F5883A09F403C2893A09F034
:1039300006CFC32DC17080910F01909110010E949C
:10394000E633A82E682F822D0E94A21980910F01C4
:103950009091100101979093100180930F01209195
:103960001801309119012150310930931901209328
:103970001801832D8E7F9FC1803B09F40DC208F092
:1039800039C28B3A09F0DBCE80910F019091100182
:103990000E94E633682FA82E8091180190E00E94C3
:1039A0003B34F4C18A3B09F4C5C240F5883B09F4B5
:1039B00069C208F096C2833B09F0C1CE80910F0125
:1039C000909110010E94E633682FA82E8091180173
:1039D00090E00E943B3480910F019091100101967C
:1039E0009093100180930F01809119018150809371
:1039F00019018111E3CF832D82648ACF8C3F09F4B2
:103A0000B7C28D3F09F4BBC28B3B09F098CE8091C1
:103A10000F01909110010E94E633682FA82E80912B
:103A2000180190E00E943B3480910F0190911001A9
:103A300001979093100180930F018091190181509B
:103A4000809319018111E3CF932D926448C2809134
:103A5000180190E00E94283480931901932DE82FDB
:103A6000F0E0E051FF4FE4919B73E92BED7E3E2E99
:103A700029C0809118016091190190E00E943B34A7
:103A800021C0609118017091190180910F019091EE
:103A900010018DC00E941F184C01609118010E94F6
:103AA0001A3460911901C40101960E941A340AC0A7
:103AB000622D80E00E94A219A82E222031F0689485
:103AC00030F8282ECF91FF900895E89430F8F9CF80
:103AD00010921601F7CF20921401F4CF80911801B3
:103AE000682FCBCF609118017091190180910F015F
:103AF000909110010E9460199093100180930F0122
:103B0000E1CF0E941F184C010E94E63380931801F8
:103B1000C40101960E94E63380931901D3CF20920D
:103B20001301D0CF8091180190E00E942834809337
:103B30001B0194CF60911A0170911B01A6CF81E007
:103B400080931601BFCFE09114012E2E832DF0E05B
:103B5000E051FF4FE4918B73E82B3E2E80911501CD
:103B60008823B1F0E46083CF8091180190E00E9437
:103B7000283480931A0172CF8091180160911A0144
:103B80007CCF60911A0170911B01B0CF82E0D8CF39
:103B9000EB7F6DCF8091180190E00E9428348093D4
:103BA00010015CCF80910F0190911001BC010E9427
:103BB000F519A2CF80910F01909110010E94E63378
:103BC000722D682F4B01822D807F282E862F8F70BB
:103BD000282A34E0769567953A95E1F7A62E8091EC
:103BE0000F01909110010E941A34832DE22DF0E014
:103BF000E051FF4FE4918B73E82B38CF809118018F
:103C000060910F013ACF80910F01909110010E94B5
:103C1000E633922D4C0124E0969587952A95E1F79D
:103C20008F70922D907F292E282A692D6F70882DF4
:103C30008295807F682BD2CFB30127CF0E941F18B7
:103C40004C01662D0E941A34672D2DCF622D809174
:103C5000180113CFB3014ACF0E941F184C010E94D4
:103C6000E633682E712CC40101960E94E633782A4F
:103C700029CF80910F01909110010E94E633A82E68
:103C8000C32D682F822D0E94A21980910F0190915F
:103C9000100101969093100180930F01209118015B
:103CA00030911901215031093093190120931801E5
:103CB000832D8E7FC1708C2BF82E6894F1F83F2CE9
:103CC000232B09F035C18B7F24C08091180190E02F
:103CD0000E942834A82E682F80910F019091100126
:103CE0000E941A3480910F019091100101969093D7
:103CF000100180930F019091190191509093190137
:103D0000832DF32C6894F1F83F2C992309F474CE99
:103D10008F7B8260FDCD80910F01909110010E94F8
:103D2000E633682FA82E8091180190E00E943B3462
:103D3000D9CF80910F01909110010E94E633A82EF7
:103D4000682F80911A0190911B010E941A34809172
:103D50000F019091100101979093100180930F0132
:103D600080911A0190911B010197BECD689432F8A1
:103D7000CDCD8091180190E00E942834A82E682FA4
:103D800080910F01909110010E941A3480910F01CF
:103D9000909110010197ABCF80910F01909110018C
:103DA0000E94E633A82E682F80911A0190911B0182
:103DB0000E941A3480910F01909110010196909306
:103DC000100180930F0180911A0190911B010196BF
:103DD00090931B0180931A01809118019091190111
:103DE00001979093190180931801892BA9F6832DCF
:103DF000897E8ECDC32DC17080910F0190911001ED
:103E00000E94E633A82E682F822D0E94A21980916D
:103E10000F019091100101969093100180930F0172
:103E20002091180130911901215031093093190165
:103E3000209318012115310509F49BCD36FEDCCF06
:103E400098CD8091180190E00E942834A82E682F08
:103E500080910F01909110010E941A3480910F01FE
:103E60009091100101969093100180930F01809121
:103E700019018150809319018111E3CF832D8D7F2A
:103E8000806446CD80910F01909110010E94E6332D
:103E9000A82E682F80911A0190911B010E941A345C
:103EA00080910F01909110010197909310018093E0
:103EB0000F0180911A0190911B01019790931B01B2
:103EC00080931A01809118019091190101979093A4
:103ED000190180931801892BA9F6932D997E392E0B
:103EE000F1CDC32DC17080910F01909110010E94FE
:103EF000E633A82E682F822D0E94A21980910F010F
:103F00009091100101979093100180930F012091DF
:103F10001801309119012150310930931901209372
:103F200018012115310509F424CD36FEDCCF21CD51
:103F30008660EECC8091180190E00E942834A82E73
:103F4000682F80910F01909110010E941A34809186
:103F50000F019091100101979093100180930F0130
:103F6000809119018150809319018111E3CF43CDD4
:103F700080910F01909110010E94AB34A3CD8091EC
:103F80000F01909110010E94AA349CCD0F931F93B2
:103F9000CF93DF930E941718D82F0E941718C82FAD
:103FA00000911C0110911D010D0F111DD7FD1A95D7
:103FB000C8010E94E633682FCE3709F40FC108F01C
:103FC0005AC0CE3309F4E7C088F5CE3109F4BEC03B
:103FD000E0F4CE3009F48FC0C63109F4A0C0C63079
:103FE00009F07AC0832D8C7E67FD83C0382E932D17
:103FF000832D8170660F682BE62FF0E0E051FF4FB4
:10400000E4919B739E2B392E70C0CE3209F4ACC064
:10401000C63309F4B6C0C63209F05EC0832D8C7E6B
:1040200067FDA0C0382E660F932DE6CFCE3509F47C
:10403000C6C0A0F4CE3409F4B7C0C63509F4BAC07E
:10404000C63409F049C0832D8D7B60FFB1C080610B
:10405000382EDF91CF911F910F910895CE3609F43C
:10406000B3C0C63709F4B5C0C636B1F5832D8D7B14
:1040700064FF9EC0ECCFCE3B09F4BFC0C0F4CE3984
:1040800009F4B5C050F4CE3809F4ADC0C63909F40E
:10409000ACC0C63809F56E7F28C0CE3A09F4A9C075
:1040A000C63B09F4A8C0C63AB9F46F7E1EC0CE3D27
:1040B00009F4A9C050F4CE3C09F4A1C0C63D09F4EE
:1040C000A0C0C63C49F4616010C0CE3E09F49DC05A
:1040D00030F46061C63E49F00E943C34BACFC63F1E
:1040E00009F495C06068CE3FB9F7C8010E941A3440
:1040F000B0CF81607BCF832D8C7E60FD0EC0382ECB
:104100006695832D30FC6068E62FF0E0E051FF4FAC
:10411000E4918B738E2B382EE8CF8160F0CF932DF6
:10412000232D2D7E322E880F392F3170832B67FF80
:1041300016C02160322E932DE82FF0E0E051FF4FA2
:10414000E4919B739E2B392E682FCFCF932D232D77
:104150002D7E322E869590FD806860FDEACF9C7E94
:10416000392EE9CF81605ECF832D8C7E60FD07C044
:10417000382E862F80786695682B832DC5CF816079
:10418000F7CF832D8C7E67FD04C0382E660F6160EB
:10419000F4CF8160FACF832D8C7E60FD03C0382E72
:1041A000669542CF8160FBCF832D8D7B61FD4FCF24
:1041B00080654ECF832D8D7B62FFFACF48CF832D54
:1041C0008D7B63FFF5CF43CF832D8D7B65FFF0CFD4
:1041D0003ECF832D8D7B66FFEBCF39CF832D8D7B3B
:1041E00067FFE6CF34CF6D7F80CF6B7F7ECF677F59
:1041F0007CCF6F7D7ACF6F7B78CF6F7776CF626021
:1042000074CF646072CF686070CF60626ECF60649C
:104210006CCFCF930E941718A82E8950813F08F0C9
:10422000A9C3E82FF0E0E95EFE4D0C941D3808228A
:10423000BA24BA24BA24BA24BA24BA24BA24BA248E
:10424000BA24BA24BA24BA24BA24BA24BA24172223
:10425000BA24BA24BA24BA24BA24BA24BA241C220E
:104260001F222D2233223A223F22BA24BA2442228C
:10427000482254225A2261226622BA24BA24BA243D
:10428000BA24BA2469227F229222BA24BA24A22212
:10429000BA24BA24BA24BA24BA24BA24BA24BA242E
:1042A000BA24BA24A422AB22AE22BA24BA24BA2455
:1042B000BA24BA24BD22C222C522BA24BA24BA24FE
:1042C000BA24BA24D422D922DC22BA24BA24BA24A9
:1042D000BA24BA24EB22F022F322BA2402230523C3
:1042E00008230B23A8220E2311232223252328236E
:1042F0002B232E233123A82234234523482357235D
:104300006023692372237B23BA248423BA24BA242A
:10431000BA24BA248C238F239223A822BA24BA2445
:10432000BA24BA24A223A823AB23BA24BA24BA24D9
:10433000BA24BA24BB23C123C423BA24BA24BA247E
:10434000BA24BA24D423DA23DD23BA24BA24BA2423
:10435000BA24BA24ED23F323F623BA24BA24BA24C8
:10436000BA24BA24062415241824BA24BA24BA2458
:10437000BA24BA2431243E244124BA24BA24BA24CB
:10438000BA24BA245A245E246124BA24BA24BA2452
:10439000BA24BA24712477247A24BA24BA24BA24F9
:1043A000BA24BA24BA24BA24BA24BA24BA24BA241D
:1043B000BA248A24BA24BA24BA24BA24BA24BA243D
:1043C000BA24BA24BA24BA24BA24BA24BA24BA24FD
:1043D000BA24BA24BA24BA24BA24BA24BA248D241A
:1043E000BA249024BA24A924BA24BA24BA24B02422
:1043F000BA24BA24BA24BA24BA24BA24BA24BA24CD
:10440000BA24BA24BA24BA24BA24BA24BA24B524C1
:10441000609118017091190180911C0190911D010A
:104420000E94301990931D0180931C0191C06091EE
:104430001A0170911B01F0CF0E941F18F3CF0E9448
:104440001F184C0160911C010E941A3460911D01DB
:10445000C40101960E941A347BC080911C01909186
:104460001D010196DFCF80911D010E94AA18809343
:104470001D016EC080911D010E94C418F8CF0E94DA
:104480001718F5CF80911C0190911D01BC01C8CF78
:104490000E941F184C010E94E63380931C01C40146
:1044A00001960E94E633E3CF80911C0190911D019B
:1044B0000197B8CF80911C010E94AA1880931C011B
:1044C00047C080911C010E94C418F8CF0E941718A1
:1044D000F5CF0E94171820911C0130911D01A901F0
:1044E000480F511D87FD5A95CA014A010E94E633C3
:1044F000A82E0E94AA18A82E682FC401ABCF0E9434
:10450000171820911C0130911D01A901480F511D60
:1045100087FD5A95CA014A010E94E633A82E0E94DF
:10452000C418E9CF0E941718C82F0E941718682FC7
:10453000A82E80911C0190911D018C0F911DC7FD2B
:104540009A9588CFB30168CF80911D01809319019E
:1045500081E0CF91089580911C01F8CF0E94171837
:1045600020911C0130911D01A901480F511D87FDAB
:104570005A95CA010E94E633E9CF80911D018093CC
:104580001801E6CF80911C01FACF0E9417182091E4
:104590001C0130911D01A901480F511D87FD5A953D
:1045A000CA010E94E633EBCF80911D0180931B016D
:1045B000CFCF80911C01FACF0E94171820911C01C7
:1045C00030911D01A901480F511D87FD5A95CA015F
:1045D0000E94E633EBCF80911D0180931A01B8CF82
:1045E00080911C01FACF0E94171820911C01309174
:1045F0001D01A901480F511D87FD5A95CA010E944E
:10460000E633EBCF8091190132CF809118012FCF83
:1046100080911B012CCF80911A0129CF80911C0120
:1046200026CF0E94171820911C0130911D01A9016D
:10463000480F511D87FD5A95CA010E94E6338093A9
:10464000100186CF20921D0183CF8091190136CFB2
:104650008091180133CF80911B0130CF80911A01D6
:104660002DCF80911D012ACF0E94171820911C0187
:1046700030911D01A901480F511D87FD5A95CA01AE
:104680000E94E63380930F0163CF20921C0160CF1C
:104690000E94171820911C0130911D016091190191
:1046A000A901480F511D87FD5A95CA01D3CE0E941A
:1046B000171820911C0130911D0160911801F0CF55
:1046C0000E94171820911C0130911D0160911B015F
:1046D000E7CF0E94171820911C0130911D016091B5
:1046E0001A01DECF0E94171820911C0130911D0184
:1046F00060911001D5CF0E94171820911C013091B4
:104700001D0160910F01CCCF0E941718622D2091DE
:104710001C0130911D01C4CF20901D0119CF2090A4
:104720001C0116CF0E94171820911C0130911D0109
:10473000A901480F511D87FD5A95CA010E94E63311
:10474000282E06CF60911D01822D0E94DE18F8CF21
:1047500060911C01F9CF0E94171820911C01309123
:104760001D01A901480F511D87FD5A95CA010E94DC
:10477000E633682FE9CF60911D01822D0E94051953
:10478000DFCF60911C01F9CF0E94171820911C0106
:1047900030911D01A901480F511D87FD5A95CA018D
:1047A0000E94E633682FE9CF60911D01822D0E949F
:1047B000A219C6CF60911C01F9CF0E941718209151
:1047C0001C0130911D01A901480F511D87FD5A950B
:1047D000CA010E94E633682FE9CF60911D01822D46
:1047E0000E94C919ADCF60911C01F9CF0E94171822
:1047F00020911C0130911D01A901480F511D87FD19
:104800005A95CA010E94E633682FE9CFE0911D0155
:10481000E2212E2E832DF0E0E051FF4FE4918B73C7
:10482000E82BEC7FE0613E2E93CEE0911C01F0CFAF
:104830000E94171820911C0130911D01A901480FF9
:10484000511D87FD5A95CA010E94E6338221282E08
:10485000932DE82FF0E0E051FF4FE4919B73E92B9B
:10486000E0CFE0911D01E2252E2E832DF0E0E051F6
:10487000FF4FE4918B73E82BEC7ED5CFE0911C01C8
:10488000F2CF0E94171820911C0130911D01A9013F
:10489000480F511D87FD5A95CA010E94E6338225B3
:1048A000282E932DE82FF0E0E051FF4FE4919B7309
:1048B000E92BE2CFE0911D01E229D6CFE0911C0166
:1048C000FBCF0E94171820911C0130911D01A901F6
:1048D000480F511D87FD5A95CA010E94E63382296F
:1048E000DFCF60911D01822D0E94A21931CE60910F
:1048F0001C01F9CF0E94171820911C0130911D0155
:10490000A901480F511D87FD5A95CA010E94E6333F
:10491000682FE9CF0E94C61F1BCE0E94481882CD87
:10492000C3010E94E633A82E60911C01C3010E94BE
:104930001A34A0921C01C30101960E94E633A82EEE
:1049400060911D01C30101960E941A34A0921D01BD
:10495000FFCD80911C0190911D010E943818F8CD67
:1049600040901C0150901D01F3CD60901C0170908F
:104970001D01EECD80E0EDCD0F931F93CF93DF931C
:104980000E941718D82F0E941718C82F00911101E4
:10499000109112010D0F111DD7FD1A95C8010E942B
:1049A000E633682FCE3709F40FC108F05AC0CE3372
:1049B00009F4E7C088F5CE3109F4BEC0E0F4CE308A
:1049C00009F48FC0C63109F4A0C0C63009F07AC01E
:1049D000832D8C7E67FD83C0382E932D832D8170AF
:1049E000660F682BE62FF0E0E051FF4FE4919B73D8
:1049F0009E2B392E70C0CE3209F4ACC0C63309F4F8
:104A0000B6C0C63209F05EC0832D8C7E67FDA0C0A3
:104A1000382E660F932DE6CFCE3509F4C6C0A0F42C
:104A2000CE3409F4B7C0C63509F4BAC0C63409F0AB
:104A300049C0832D8D7B60FFB1C08061382EDF912E
:104A4000CF911F910F910895CE3609F4B3C0C637A8
:104A500009F4B5C0C636B1F5832D8D7B64FF9EC0C9
:104A6000ECCFCE3B09F4BFC0C0F4CE3909F4B5C0D9
:104A700050F4CE3809F4ADC0C63909F4ACC0C6381C
:104A800009F56E7F28C0CE3A09F4A9C0C63B09F4E7
:104A9000A8C0C63AB9F46F7E1EC0CE3D09F4A9C0C5
:104AA00050F4CE3C09F4A1C0C63D09F4A0C0C63CF8
:104AB00049F4616010C0CE3E09F49DC030F46061DD
:104AC000C63E49F00E943C34BACFC63F09F495C0B7
:104AD0006068CE3FB9F7C8010E941A34B0CF816038
:104AE0007BCF832D8C7E60FD0EC0382E6695832D86
:104AF00030FC6068E62FF0E0E051FF4FE4918B73EB
:104B00008E2B382EE8CF8160F0CF932D232D2D7E74
:104B1000322E880F392F3170832B67FF16C021602A
:104B2000322E932DE82FF0E0E051FF4FE4919B737C
:104B30009E2B392E682FCFCF932D232D2D7E322EF5
:104B4000869590FD806860FDEACF9C7E392EE9CF86
:104B500081605ECF832D8C7E60FD07C0382E862F4E
:104B600080786695682B832DC5CF8160F7CF832D24
:104B70008C7E67FD04C0382E660F6160F4CF8160C3
:104B8000FACF832D8C7E60FD03C0382E669542CF10
:104B90008160FBCF832D8D7B61FD4FCF80654ECF34
:104BA000832D8D7B62FFFACF48CF832D8D7B63FFF2
:104BB000F5CF43CF832D8D7B65FFF0CF3ECF832D87
:104BC0008D7B66FFEBCF39CF832D8D7B67FFE6CFE3
:104BD00034CF6D7F80CF6B7F7ECF677F7CCF6F7D43
:104BE0007ACF6F7B78CF6F7776CF626074CF646057
:104BF00072CF686070CF60626ECF60646CCFCF930D
:104C00000E941718A82E8950813F08F0A9C3E82FE9
:104C1000F0E0E35FF94D0C941D38FE26B029B02971
:104C2000B029B029B029B029B029B029B029B029BC
:104C3000B029B029B029B029B0290D27B029B02951
:104C4000B029B029B029B029B02912271527232768
:104C5000292730273527B029B02938273E274A276A
:104C6000502757275C27B029B029B029B029B0298F
:104C70005F2775278827B029B0299827B029B02940
:104C8000B029B029B029B029B029B029B029B0295C
:104C90009A27A127A427B029B029B029B029B02983
:104CA000B327B827BB27B029B029B029B029B0292C
:104CB000CA27CF27D227B029B029B029B029B029D7
:104CC000E127E627E927B029F827FB27FE27012857
:104CD0009E270428072818281B281E282128242856
:104CE00027289E272A283B283E284D2856285F281B
:104CF00068287128B0297A28B029B029B029B029AC
:104D00008228852888289E27B029B029B029B02973
:104D100098289E28A128B029B029B029B029B02907
:104D2000B128B728BA28B029B029B029B029B029AC
:104D3000CA28D028D328B029B029B029B029B02951
:104D4000E328E928EC28B029B029B029B029B029F6
:104D5000FC280B290E29B029B029B029B029B02987
:104D6000272934293729B029B029B029B029B029F9
:104D7000502954295729B029B029B029B029B02980
:104D800067296D297029B029B029B029B029B02927
:104D9000B029B029B029B029B029B029B02980297B
:104DA000B029B029B029B029B029B029B029B0293B
:104DB000B029B029B029B029B029B029B029B0292B
:104DC000B029B029B029B029B0298329B029862972
:104DD000B0299F29B029B029B029A629B029B02926
:104DE000B029B029B029B029B029B029B029B029FB
:104DF000B029B029B029B029B029AB296091180198
:104E00007091190180911101909112010E94301945
:104E1000909312018093110191C060911A017091D9
:104E20001B01F0CF0E941F18F3CF0E941F184C01E6
:104E3000609111010E941A3460911201C40101961F
:104E40000E941A347BC08091110190911201019649
:104E5000DFCF809112010E94AA18809312016EC0C8
:104E6000809112010E94C418F8CF0E941718F5CF44
:104E70008091110190911201BC01C8CF0E941F18AE
:104E80004C010E94E63380931101C40101960E94F7
:104E9000E633E3CF80911101909112010197B8CFD1
:104EA000809111010E94AA188093110147C080913E
:104EB00011010E94C418F8CF0E941718F5CF0E9464
:104EC00017182091110130911201A901480F511DAD
:104ED00087FD5A95CA014A010E94E633A82E0E9416
:104EE000AA18A82E682FC401ABCF0E9417182091D2
:104EF000110130911201A901480F511D87FD5A95EA
:104F0000CA014A010E94E633A82E0E94C418E9CFC4
:104F10000E941718C82F0E941718682FA82E80917A
:104F20001101909112018C0F911DC7FD9A9588CFA8
:104F3000B30168CF809112018093190181E0CF9174
:104F4000089580911101F8CF0E9417182091110146
:104F500030911201A901480F511D87FD5A95CA01D0
:104F60000E94E633E9CF8091120180931801E6CFC9
:104F700080911101FACF0E941718209111013091F0
:104F80001201A901480F511D87FD5A95CA010E94BF
:104F9000E633EBCF8091120180931B01CFCF80913C
:104FA0001101FACF0E9417182091110130911201BE
:104FB000A901480F511D87FD5A95CA010E94E63389
:104FC000EBCF8091120180931A01B8CF809111012B
:104FD000FACF0E9417182091110130911201A901F6
:104FE000480F511D87FD5A95CA010E94E633EBCF49
:104FF0008091190132CF809118012FCF80911B0130
:105000002CCF80911A0129CF8091110126CF0E94C7
:1050100017182091110130911201A901480F511D5B
:1050200087FD5A95CA010E94E6338093100186CF0E
:105030002092120183CF8091190136CF80911801FF
:1050400033CF80911B0130CF80911A012DCF8091F9
:1050500012012ACF0E9417182091110130911201DC
:10506000A901480F511D87FD5A95CA010E94E633D8
:1050700080930F0163CF2092110160CF0E94171817
:10508000209111013091120160911901A901480F7D
:10509000511D87FD5A95CA01D3CE0E941718209141
:1050A00011013091120160911801F0CF0E94171880
:1050B000209111013091120160911B01E7CF0E94F4
:1050C0001718209111013091120160911A01DECF61
:1050D0000E94171820911101309112016091100166
:1050E000D5CF0E94171820911101309112016091C3
:1050F0000F01CCCF0E941718622D20911101309121
:105100001201C4CF2090120119CF2090110116CFA7
:105110000E9417182091110130911201A901480F26
:10512000511D87FD5A95CA010E94E633282E06CFED
:1051300060911201822D0E94DE18F8CF609111015A
:10514000F9CF0E9417182091110130911201A90185
:10515000480F511D87FD5A95CA010E94E633682FFA
:10516000E9CF60911201822D0E940519DFCF609175
:105170001101F9CF0E9417182091110130911201ED
:10518000A901480F511D87FD5A95CA010E94E633B7
:10519000682FE9CF60911201822D0E94A219C6CF1B
:1051A00060911101F9CF0E941718209111013091DF
:1051B0001201A901480F511D87FD5A95CA010E948D
:1051C000E633682FE9CF60911201822D0E94C91940
:1051D000ADCF60911101F9CF0E94171820911101F4
:1051E00030911201A901480F511D87FD5A95CA013E
:1051F0000E94E633682FE9CFE0911201E2212E2EC2
:10520000832DF0E0E051FF4FE4918B73E82BEC7FAE
:10521000E0613E2E93CEE0911101F0CF0E9417186D
:105220002091110130911201A901480F511D87FDF4
:105230005A95CA010E94E6338221282E932DE82F29
:10524000F0E0E051FF4FE4919B73E92BE0CFE09158
:105250001201E2252E2E832DF0E0E051FF4FE49164
:105260008B73E82BEC7ED5CFE0911101F2CF0E9439
:1052700017182091110130911201A901480F511DF9
:1052800087FD5A95CA010E94E6338225282E932D68
:10529000E82FF0E0E051FF4FE4919B73E92BE2CF60
:1052A000E0911201E229D6CFE0911101FBCF0E94DB
:1052B00017182091110130911201A901480F511DB9
:1052C00087FD5A95CA010E94E6338229DFCF60919B
:1052D0001201822D0E94A21931CE60911101F9CFE5
:1052E0000E9417182091110130911201A901480F55
:1052F000511D87FD5A95CA010E94E633682FE9CFF8
:105300000E94BC241BCE0E94481882CDC3010E947B
:10531000E633A82E60911101C3010E941A34A092B5
:105320001101C30101960E94E633A82E609112017B
:10533000C30101960E941A34A0921201FFCD809100
:105340001101909112010E943818F8CD409011017E
:1053500050901201F3CD6090110170901201EECDCA
:1053600080E0EDCDCF930E941718A82E80911301F5
:105370008F5F80931301EA2DF0E0EF53F64D0C940C
:105380001D38C72AC12AC92AD12ADB2AE22AE92ADA
:10539000EE2AFF2A0C2B1B2B232B2D2B342B3B2BE4
:1053A000402B522B642B6B2B732B7D2B842B8B2B45
:1053B000902BA32BAA2BB92BC12BCB2BD22BD92BC8
:1053C000DE2BF32BFF2B062C142C1E2C252C2C2C27
:1053D000312C342C402C4C2C5A2C642C6B2C722CE1
:1053E000772C7C2C882C8C2C932C972CA92CBB2CC8
:1053F000C62CCB2CD72CE32CEA2CEE2CF32CF82C3F
:10540000FC2CC72A062D0B2D102D152D1A2D1F2D06
:10541000282D2B2DC72A302D352D3A2D3F2D442DEB
:105420004D2D502D552DC72A5A2D5F2D642D692DD8
:10543000722D752D7A2D7F2DC72A842D892D8E2DC5
:10544000972D9A2D9F2DA42DA92DC72AAE2DB32DB2
:10545000BC2DBF2DC42DC92DCE2DD32DC72AD82D9F
:10546000E12DE42DED2DF62DFF2D082E112E1A2EF7
:105470001E2E262E292E2C2E2F2E322E352E382E55
:10548000C72A402E472E4E2E552E5C2E632E6A2E96
:10549000762E7C2E832E8A2E912E982E9F2EA62E2F
:1054A000B22EB82EBF2EC62ECD2ED42EDB2EE22E3F
:1054B000EE2EF42EFB2E022F092F102F172F1E2F4A
:1054C0002A2F302F3F2F4E2F5D2F6C2F7B2F8A2FAF
:1054D0009E2FAA2FB82FC62FD42FE22FF02FFE2FEA
:1054E00011301B30293037304530533061306F3048
:1054F00082308D30933099309F30A530AB30B13051
:10550000BC30C130C730CE30D530D930E330EA308E
:10551000F330F930FC30003107310A3114311C31DD
:1055200025312C312F3136313D3145314F31563116
:105530005F31663169319B31A231AA31B431BB315F
:10554000C431CB31CE31D531DC31F63100320732C6
:1055500018321F32223227322E3240324A324D3236
:105560005D32643267326E3276327C328932913209
:10557000A232AA32AF32B532BF32C632D332D632BD
:10558000DF320E941F189093190180931801CF9168
:105590000895622D80911801909119010E941A348A
:1055A000F6CF8091180190911901019690931901FD
:1055B00080931801ECCF809119010E94AA18809362
:1055C0001901E5CF809119010E94C4188093190137
:1055D000DECF0E94171880931901D9CF822DA22CFB
:1055E000222D220F211D222E87FF06C0689430F83D
:1055F000332D3D7E332ECBCFE89430F8F9CF822D7A
:10560000A22C2090090180930901832DA32C3090B6
:105610001E0180931E01BBCF60911801709119018A
:1056200080910F01909110010E9430199093100108
:1056300080930F01ACCF80911801909119010E94C5
:10564000E633282EA4CF809118019091190101977B
:1056500090931901809318019ACF809118010E94AC
:10566000AA188093180193CF809118010E94C41842
:10567000809318018CCF0E9417188093180187CF50
:10568000822DA22C922D90FB979597F9292E80FFC1
:1056900006C0689430F8232D2D7E322E78CFE89402
:1056A00030F8F9CF0E9417189201280F311D87FD9D
:1056B0003A954901809119018150809319018823FD
:1056C00009F465CF290163CF0E941F1890931B0135
:1056D00080931A015CCF622D80911A0190911B0179
:1056E0000E941A3454CF80911A0190911B010196A7
:1056F00090931B0180931A014ACF80911B010E9455
:10570000AA1880931B0143CF80911B010E94C418EB
:1057100080931B013CCF0E94171880931B0137CF49
:10572000822DA22C322D330F232E932D9170292AF6
:1057300087FF06C0689430F8832D8D7E382E27CFE2
:10574000E89430F8F9CF0E941718480E511C87FDD5
:105750005A941DCF60911A0170911B0180910F0125
:10576000909110010E9430199093100180930F01C5
:105770000ECF80911A0190911B010E94E633282ED2
:1057800006CF80911A0190911B01019790931B0104
:1057900080931A01FCCE80911A010E94AA1880936E
:1057A0001A01F5CE80911A010E94C41880931A0143
:1057B000EECE0E94171880931A01E9CE822DA22CFA
:1057C000922D9695292E90E8399E90011124222A37
:1057D00080FF06C0689430F8232D2D7E322ED7CE60
:1057E000E89430F8F9CF0E9417189201280F311D64
:1057F00087FD3A95490136FCCACE2901C8CE0E94E0
:105800001F189093100180930F01C1CE0E941F18A2
:105810004C0160910F010E941A3460911001C40183
:1058200001960E941A34B3CE80910F01909110011D
:1058300001969093100180930F01A9CE80911001E1
:105840000E94AA1880931001A2CE809110010E949C
:10585000C418809310019BCE0E94171880931001EA
:1058600096CE0E94641893CE0E9417189201280FBA
:10587000311D87FD3A95490136FE89CE290187CE33
:1058800080910F0190911001BC010E9430199093FA
:10589000100180930F017BCE0E941F184C010E94C3
:1058A000E63380930F01C40101960E94E633809392
:1058B00010016DCE80910F0190911001019790938E
:1058C000100180930F0163CE80910F010E94AA18EE
:1058D00080930F015CCE80910F010E94C4188093C9
:1058E0000F0155CE0E94171880930F0150CE2094BF
:1058F000332D3261332E4BCE0E9417189201280FA0
:10590000311D87FD3A95490130FC41CE29013FCE3A
:105910000E941F183C013BCE0E941F184C01622DB3
:105920000E941A3434CE3FEF631A730A30CE80914E
:105930000F01909110010E94E633A82E0E94AA1830
:10594000A82E682F80910F01909110010E941A34A7
:105950001ECE80910F01909110010E94E633A82E77
:105960000E94C418A82E682F80910F0190911001F9
:105970000E941A340CCE0E941718A82E682F80910E
:105980000F01909110010E941A3401CE832D8D7E5B
:105990008160382EFCCD0E9417189201280F311D0E
:1059A00087FD3A95490130FEF2CD2901F0CDB301D2
:1059B00080910F01909110010E9430199093100175
:1059C00080930F01E4CD0E941F184C010E94E63322
:1059D000282EDDCD31E0631A7108D9CD822D0E94C9
:1059E000AA18282ED4CD822D0E94C418282ECFCDDF
:1059F0000E941718282ECBCD832D8D7E30FC04C03D
:105A0000382E81E03826C3CD8061FACF809118010D
:105A100080931901BCCD80911B0180931901B7CDF2
:105A200080911A0180931901B2CD80911001809369
:105A30001901ADCD80910F0180931901A8CD8091FE
:105A40000F01909110010E94E633809319019FCDC0
:105A5000209219019CCD809119018093180197CD56
:105A600080911B018093180192CD80911A0180933F
:105A700018018DCD809110018093180188CD8091FF
:105A80000F018093180183CD80910F019091100137
:105A90000E94E633809318017ACD2092180177CDC9
:105AA0008091190180931B0172CD80911801809320
:105AB0001B016DCD80911A0180931B0168CD8091EF
:105AC000100180931B0163CD80910F0180931B0116
:105AD0005ECD80910F01909110010E94E63380937A
:105AE0001B0155CD20921B0152CD8091190180934D
:105AF0001A014DCD8091180180931A0148CD8091F3
:105B00001B0180931A0143CD8091100180931A01EB
:105B10003ECD80910F0180931A0139CD80910F0104
:105B2000909110010E94E63380931A0130CD2092AB
:105B30001A012DCD809119018093100128CD8091FB
:105B400018018093100123CD80911B0180931001D7
:105B50001ECD80911A018093100119CD80910F0103
:105B60008093100114CD80910F01909110010E943B
:105B7000E633809310010BCD2092100108CD809167
:105B8000190180930F0103CD8091180180930F01BB
:105B9000FECC80911B0180930F01F9CC80911A01FA
:105BA00080930F01F4CC8091100180930F01EFCC12
:105BB00080910F01909110010E94E63380930F01B4
:105BC000E6CC20920F01E3CC6091190180910F0186
:105BD000909110010E941A34DACC609118018091E2
:105BE0000F01909110010E941A34D1CC60911B01D9
:105BF00080910F01909110010E941A34C8CC6091DD
:105C00001A0180910F01909110010E941A34BFCCAB
:105C10006091100180910F01909110010E941A343F
:105C2000B6CC60910F0180910F01909110010E94FC
:105C30001A34ADCC81E080931701A9CC622D8091FC
:105C40000F01909110010E941A34A1CC20901901EB
:105C50009ECC209018019BCC20901B0198CC2090CA
:105C60001A0195CC2090100192CC20900F018FCC7E
:105C700080910F01909110010E94E633282E87CC6D
:105C800060911901822D0E94DE18282E80CC60912F
:105C90001801822D0E94DE18282E79CC60911B01FC
:105CA000822D0E94DE18282E72CC60911A01822D5E
:105CB0000E94DE18282E6BCC60911001822D0E946C
:105CC000DE18282E64CC60910F01822D0E94DE1810
:105CD000282E5DCC80910F01909110010E94E63337
:105CE000682F822D0E94DE18282E51CC822D622D25
:105CF0000E94DE18282E4BCC60911901822D0E9443
:105D00000519282E44CC60911801822D0E94051996
:105D1000282E3DCC60911B01822D0E940519282E52
:105D200036CC60911A01822D0E940519282E2FCCA5
:105D300060911001822D0E940519282E28CC6091B7
:105D40000F01822D0E940519282E21CC80910F0170
:105D5000909110010E94E633682F822D0E94051950
:105D6000282E15CC822D622D0E940519282E0FCCCD
:105D700060911901822D0E94A219282E08CC6091F1
:105D80001801822D0E94A219282E01CC60911B01BE
:105D9000822D0E94A219282EFACB60911A01822D21
:105DA0000E94A219282EF3CB60911001822D0E942F
:105DB000A219282EECCB60910F01822D0E94A2190E
:105DC000282EE5CB80910F01909110010E94E633BF
:105DD000682F822D0E94A219282ED9CB822D622DE8
:105DE0000E94A219282ED3CB60911901822D0E9406
:105DF000C919282ECCCB60911801822D0E94C91997
:105E0000282EC5CB60911B01822D0E94C919282E16
:105E1000BECB60911A01822D0E94C919282EB7CBE2
:105E200060911001822D0E94C919282EB0CB60917B
:105E30000F01822D0E94C919282EA9CB80910F0134
:105E4000909110010E94E633682F822D0E94C9199B
:105E5000282E9DCB822D622D0E94C919282E97CB0A
:105E6000E0911901E2212E2E832DF0E0E051FF4F49
:105E7000E4918B73E82BEC7FE0613E2E88CBE091C0
:105E80001801E2212E2E832DF0E0E051FF4FE49126
:105E90008B73E82BEC7FE0613E2E79CBE0911B0108
:105EA000E2212E2E832DF0E0E051FF4FE4918B7321
:105EB000E82BEC7FE0613E2E6ACBE0911A01E221F3
:105EC0002E2E832DF0E0E051FF4FE4918B73E82BF1
:105ED000EC7FE0613E2E5BCBE0911001E2212E2EA3
:105EE000832DF0E0E051FF4FE4918B73E82BEC7FC2
:105EF000E0613E2E4CCBE0910F01E2212E2E832D4E
:105F0000F0E0E051FF4FE4918B73E82BEC7FE06110
:105F10003E2E3DCB80910F01909110010E94E633FF
:105F20008221282E932DE82FF0E0E051FF4FE491DD
:105F30009B73E92BEC7FE0613E2E29CB832DE22D74
:105F4000F0E0E051FF4FE4918B738E2B8C7F8061EA
:105F5000382E1DCBE0911901E2252E2E832DF0E085
:105F6000E051FF4FE4918B73E82BEC7E3E2E0FCB7C
:105F7000E0911801E2252E2E832DF0E0E051FF4F35
:105F8000E4918B73E82BEC7E3E2E01CBE0911B015C
:105F9000E2252E2E832DF0E0E051FF4FE4918B732C
:105FA000E82BEC7E3E2EF3CAE0911A01E2252E2E5C
:105FB000832DF0E0E051FF4FE4918B73E82BEC7EF2
:105FC0003E2EE5CAE0911001E2252E2E832DF0E051
:105FD000E051FF4FE4918B73E82BEC7E3E2ED7CA45
:105FE000E0910F01E2252E2E832DF0E0E051FF4FCE
:105FF000E4918B73E82BEC7E3E2EC9CA80910F0191
:10600000909110010E94E6338225282E932DE82FCF
:10601000F0E0E051FF4FE4919B73E92BEC7E3E2EC4
:10602000B6CA212C832DE0EFF0E0E4918B738E2B28
:106030008C7E382EACCAE0911901E2292E2E832DD8
:10604000F0E0E051FF4FE4918B73E82BEC7E3E2EA5
:106050009ECAE0911801E2292E2E832DF0E0E05136
:10606000FF4FE4918B73E82BEC7E3E2E90CAE091BB
:106070001B01E2292E2E832DF0E0E051FF4FE49129
:106080008B73E82BEC7E3E2E82CAE0911A01E22946
:106090002E2E832DF0E0E051FF4FE4918B73E82B1F
:1060A000EC7E3E2E74CAE0911001E2292E2E832D43
:1060B000F0E0E051FF4FE4918B73E82BEC7E3E2E35
:1060C00066CAE0910F01E2292E2E832DF0E0E05107
:1060D000FF4FE4918B73E82BEC7E3E2E58CA8091E3
:1060E0000F01909110010E94E6338229282E932DF2
:1060F000E82FF0E0E051FF4FE4919B73E92BEC7E39
:106100003E2E45CA832DE22DF0E0E051FF4FE49191
:106110008B73E82BEC7E3E2E3ACA60911901822DDA
:106120000E94A21934CA60911801822D0E94A219FE
:106130002ECA60911B01822D0E94A21928CA60916B
:106140001A01822D0E94A21922CA60911001822D8B
:106150000E94A2191CCA60910F01822D0E94A219EF
:1061600016CA80910F01909110010E94E633682FAA
:10617000822D0E94A2190BCA822D622D0E94A219A3
:1061800006CA36FC04CA0E9448182C0100CA0E94A4
:1061900048189093190180931801F9C90E941F189B
:1061A0004C0136FCF4C92C01F2C90E941F182C01C5
:1061B000EEC90E941F184C0136FCE9C9C2010E94B9
:1061C00038182401E4C980911801909119010E94A6
:1061D0003818DDC90E941718A82E682F822D0E943A
:1061E000DE18282ED4C9C2010E943818512C412C27
:1061F000CEC936FECCC9C7CF0E9448182C01C7C9EA
:106200000E941F184C0136FEC2C92C01C0C90E9451
:10621000371ABDC90E941F184C0136FEB8C9C20109
:106220000E9438182401B3C90E941F184C01C201F2
:106230000E9438182401ABC90E941718A82E682F95
:10624000822D0E940519282EA2C9C2010E94381869
:1062500068E0462E512C9BC930FC99C994CF0E940E
:10626000481890931B0180931A0191C90E941F182E
:106270004C0130FC8CC92C018AC90E941718A82E29
:10628000622D90E00E943B3482C90E941F184C018D
:1062900030FC7DC9C2010E943818240178C9809160
:1062A0001A0190911B010E94381871C90E94171899
:1062B000A82E682F822D0E94A219282E68C9C2011B
:1062C0000E94381850E1452E512C61C930FE5FC93B
:1062D0005ACF809118019091190120910A013091B3
:1062E0000B01309319012093180190930B018093B7
:1062F0000A0180911A0190911B0120910C013091AB
:106300000D0130931B0120931A0190930D0180938E
:106310000C0180910F01909110014C012091070117
:10632000309108013093100120930F0190930801E0
:10633000809307012CC90E941F184C0130FE27C909
:106340002C0125C90E941718A82E90E00E9428341D
:10635000282E1DC90E941F184C0130FE18C9C20109
:106360000E943818240113C90E940921882311F4BE
:106370000C94BB290CC90E941718A82E682F822DD7
:106380000E94C919282E03C9C2010E94381848E189
:10639000442E512CFCC832FCFAC8F5CE0E94481895
:1063A0009093100180930F01F2C80E941F184C01B6
:1063B00032FCEDC82C01EBC8C3010E94E633C82FA4
:1063C000C30101960E94E633982E8C2E60910F0136
:1063D000C3010E941A3460911001C30101960E940A
:1063E0001A349092100180920F01D1C80E941F1898
:1063F0004C0132FCCCC8C2010E9438182401C7C825
:1064000080910F01909110010E943818C0C80E941D
:106410001718A82E8221282E932DE82FF0E0E051A6
:10642000FF4FE4919B73E92BEC7FE0613E2EAFC8F8
:10643000C2010E94381830E2432E512CA8C832FE07
:10644000A6C8A1CE40900F0150901001A0C80E9494
:106450001F184C0132FE9BC82C0199C880911A016B
:1064600090911B014C0120910F013091100130934C
:106470001B0120931A019093100180930F0187C88C
:106480000E941F184C0132FE82C8C2010E943818B7
:1064900024017DC80E94831B7AC80E941718A82E69
:1064A0008225282E932DE82FF0E0E051FF4FE49154
:1064B0009B73E92BEC7E3E2E6AC8C2010E943818FD
:1064C00028E2422E512C63C837FC61C85CCE0E9482
:1064D0003018382E0E943018282E59C80E941F18D4
:1064E0004C0137FC54C82C010C94C72A109215019A
:1064F00010920E010C94C72A0E941F184C0137FEFF
:1065000002C00C94C72AC2010E94381824010C94BE
:10651000C72A822D0E942918832D0E9429180C94C5
:10652000C72A0E941718A82E8229282E932DE82FFB
:10653000F0E0E051FF4FE4919B73E92BEC7E3E2E9F
:106540000C94C72AC2010E94381890E3492E512C9E
:106550000C94C72A37FC02C00C94C72A14CE609052
:106560000F01709010010C94C72A0E941F184C0153
:1065700037FC02C00C94C72A2C010C94C72A81E076
:106580008093150180930E010C94C72A0E941F1856
:106590004C0137FC02C00C94C72AC2010E94381873
:1065A00024010C94C72A0E94FF25E0CE0E941718F0
:1065B000A82E682F822D0E94A2190C94C72AC2010E
:1065C0000E94381888E3482E512C0C94C72A0F9348
:1065D0000FB70F931F931091840004E1011B035028
:1065E000F0F7019500FF00C001FF00C001FF00C0EF
:1065F000479800E002B90F921F9211242F933F9306
:106600004F935F936F937F938F939F93AF93BF93BA
:10661000CF93DF93EF93FF9380910001909101015D
:1066200001969093010180930001109227018091BF
:106630000001909101018233914020F481E0809328
:10664000270103C000C000C000C0809100019091EC
:1066500001018533914030F0809127018F5F809355
:10666000270103C000C000C000C0809100019091CC
:1066700001018833914029F4109201011092000128
:1066800003C000C000C0000080912701882389F169
:10669000479A22E32A95F1F700C080E882B98091F9
:1066A0000001909101018134910518F18091000160
:1066B0009091010181309140E0F4809103018823A1
:1066C000C1F0809100019091010181549109F3E0A2
:1066D00096958795FA95E1F780932B1080910001AC
:1066E000909101018154877080932A100E94B734E1
:1066F0003AC08091000190910101892B51F52091C0
:106700003601203420F18091370190E0982F8827BE
:10671000865D9E4F820F911DFC0180818637B9F402
:1067200081E0809303012091650120682093650139
:106730002AE231E0A0913601B0913701BF73A20F78
:10674000B31F1196A0932901B093280102C01092A3
:10675000030180910001909101018233F1E09F07D4
:1067600011F40E94FC17FF91EF91DF91CF91BF913F
:10677000AF919F918F917F916F915F914F913F91D9
:106780002F911F900F901F910F910FBF0F91189590
:10679000F89485B7806885BF85B7806885BF8FEF1F
:1067A00081B912B83F9A8BE496E090938900809368
:1067B00088001092800089E08093810082E08093BD
:1067C0006F003E9A0E94051878940895811520E480
:1067D000920730F49F718050914FFC01849108958D
:1067E0009F738115FFE09F0728F4865D9E4FFC0193
:1067F0008081089580E0089597FD16C0811520E4FA
:10680000920730F49F718050914FFC01849108955C
:106810009F738115FFE09F0710F080E00895865D6B
:106820009E4FFC01808108959F770E94E63386FF8A
:10683000F4CF0895811520E4920748F09F738115E5
:10684000EFE09E0720F4865D9E4FFC016083089573
:1068500080FD0FC0292F30E0E0E020FD05C0F0E012
:10686000E15EFE4F8081089536952795EF5FE83011
:10687000A1F78FEF089508950895CF93DF93809146
:106880005F01282F30E0322F222780915E01820F96
:10689000932F911D009709F458C0019780935E01D2
:1068A00090935F01EFE1F1E030E020E060E070E024
:1068B00041E050E0A22F8191982F9F719F31E1F02C
:1068C000B22F211105C0982F9E7191609F3131F038
:1068D000EA0101C0CC0FAA95EAF77C2B90E08095E5
:1068E0009095880F991FA82FAE73B11104C0A6957B
:1068F000A1708C73A82B6A2B2F5F3F4F2830310576
:10690000C9F6909165019E7F862F8E7F872B49F077
:106910008091050187131CC081E02091040126139A
:1069200001C080E0892B809365017093050160931D
:106930000401709570934F0160956093500187E357
:1069400080935201DF91CF91089590E080E0A6CF2F
:1069500081E0E8CF0895E0E0F2E0A3E3B1E08491C4
:106960008D93319686E0A831B807C9F7089540E8BD
:106970002091650127FF38C32EE12A95F1F7A091F8
:106980002901B0912801F0912A1037E0F30FED9121
:10699000E6FD21C3049102B9302F3295000F02B9F0
:1069A000000FED9102B9000F00C002B9049132B995
:1069B000330F00C032B9330F00C032B9330F00C0FB
:1069C00032B9E6FD08C3000002B9302F3295000F3E
:1069D00002B9000FED9102B9000F00C002B9049195
:1069E00032B9330F00C032B9330F00C032B9330FA0
:1069F00000C032B9E6FDEFC2000002B9302F329577
:106A0000000F02B9000FED9102B9000F00C002B9EA
:106A1000049132B9330F00C032B9330F00C032B91C
:106A2000330F00C032B9E6FDD6C2000002B9302FE4
:106A30003295000F02B9000FED9102B9000F00C0AE
:106A400002B9049132B9330F00C032B9330F00C01C
:106A500032B9330F00C032B9E6FDBDC2000002B941
:106A6000302F3295000F02B9000FED9102B9000FDF
:106A700000C002B9049132B9330F00C032B9330FEC
:106A800000C032B9330F00C032B9E6FDA4C2000025
:106A900002B9302F3295000F02B9000FED9102B903
:106AA000000F00C002B9049132B9330F00C032B9EF
:106AB000330F00C032B9330F00C032B9E6FD8BC2CC
:106AC000000002B9302F3295000F02B9000FED918E
:106AD00002B9000F00C002B9049132B9330F00C0EF
:106AE00032B9330F00C032B9330F00C032B9E6FDFE
:106AF00072C2000002B9302F3295000F02B9000FA8
:106B0000ED9102B9000F00C002B9049132B9330F00
:106B100000C032B9330F00C032B9330F00C032B9F0
:106B2000E6FD59C2000002B9302F3295000F02B9BC
:106B3000000FED9102B9000F00C002B9049132B903
:106B4000330F00C032B9330F00C032B9330F00C069
:106B500032B9E6FD40C2000002B9302F3295000F75
:106B600002B9000FED9102B9000F00C002B9049103
:106B700032B9330F00C032B9330F00C032B9330F0E
:106B800000C032B9E6FD27C2000002B9302F3295AD
:106B9000000F02B9000FED9102B9000F00C002B959
:106BA000049132B9330F00C032B9330F00C032B98B
:106BB000330F00C032B9E6FD0EC2000002B9302F1B
:106BC0003295000F02B9000FED9102B9000F00C01D
:106BD00002B9049132B9330F00C032B9330F00C08B
:106BE00032B9330F00C032B9E6FDF5C1000002B979
:106BF000302F3295000F02B9000FED9102B9000F4E
:106C000000C002B9049132B9330F00C032B9330F5A
:106C100000C032B9330F00C032B9E6FDDCC100005C
:106C200002B9302F3295000F02B9000FED9102B971
:106C3000000F00C002B9049132B9330F00C032B95D
:106C4000330F00C032B9330F00C032B9E6FDC3C103
:106C5000000002B9302F3295000F02B9000FED91FC
:106C600002B9000F00C002B9049132B9330F00C05D
:106C700032B9330F00C032B9330F00C032B9E6FD6C
:106C8000AAC1000002B9302F3295000F02B9000FDF
:106C9000ED9102B9000F00C002B9049132B9330F6F
:106CA00000C032B9330F00C032B9330F00C032B95F
:106CB000E6FD91C1000002B9302F3295000F02B9F4
:106CC000000FED9102B9000F00C002B9049132B972
:106CD000330F00C032B9330F00C032B9330F00C0D8
:106CE00032B9E6FD78C1000002B9302F3295000FAD
:106CF00002B9000FED9102B9000F00C002B9049172
:106D000032B9330F00C032B9330F00C032B9330F7C
:106D100000C032B9E6FD5FC1000002B9302F3295E4
:106D2000000F02B9000FED9102B9000F00C002B9C7
:106D3000049132B9330F00C032B9330F00C032B9F9
:106D4000330F00C032B9E6FD46C1000002B9302F52
:106D50003295000F02B9000FED9102B9000F00C08B
:106D600002B9049132B9330F00C032B9330F00C0F9
:106D700032B9330F00C032B9E6FD2DC1000002B9AF
:106D8000302F3295000F02B9000FED9102B9000FBC
:106D900000C002B9049132B9330F00C032B9330FC9
:106DA00000C032B9330F00C032B9E6FD14C1000093
:106DB00002B9302F3295000F02B9000FED9102B9E0
:106DC000000F00C002B9049132B9330F00C032B9CC
:106DD000330F00C032B9330F00C032B9E6FDFBC03B
:106DE000000002B9302F3295000F02B9000FED916B
:106DF00002B9000F00C002B9049132B9330F00C0CC
:106E000032B9330F00C032B9330F00C032B9E6FDDA
:106E1000E2C0000002B9302F3295000F02B9000F16
:106E2000ED9102B9000F00C002B9049132B9330FDD
:106E300000C032B9330F00C032B9330F00C032B9CD
:106E4000E6FDC9C0000002B9302F3295000F02B92B
:106E5000000FED9102B9000F00C002B9049132B9E0
:106E6000330F00C032B9330F00C032B9330F00C046
:106E700032B9E6FDB0C0000002B9302F3295000FE4
:106E800002B9000FED9102B9000F00C002B90491E0
:106E900032B9330F00C032B9330F00C032B9330FEB
:106EA00000C032B9E6FD97C0000002B9302F32951C
:106EB000000F02B9000FED9102B9000F00C002B936
:106EC000049132B9330F00C032B9330F00C032B968
:106ED000330F00C032B9E6FD7EC0000002B9302F8A
:106EE0003295000F02B9000FED9102B9000F00C0FA
:106EF00002B9049132B9330F00C032B9330F00C068
:106F000032B9330F00C032B9E6FD65C0000002B9E6
:106F1000302F3295000F02B9000FED9102B9000F2A
:106F200000C002B9049132B9330F00C032B9330F37
:106F300000C032B9330F00C032B9E6FD4CC00000CA
:106F400002B9302F3295000F02B9000FED9102B94E
:106F5000000F00C002B9049132B9330F00C032B93A
:106F6000330F00C032B9330F00C032B9E6FD33C071
:106F7000000002B9302F3295000F02B9000FED91D9
:106F800002B9000F00C002B9049132B9330F00C03A
:106F900032B9330F00C032B9330F00C032B9E6FD49
:106FA0001AC0000002B9302F3295000F02B9000F4D
:106FB000ED9102B9000F00C002B9049132B9330F4C
:106FC00000C032B9330F00C032B9330F00C032B93C
:106FD000E6FD01C0000042B900912A10073021F4FB
:106FE000A0932901B093280108958FEF80931F018A
:106FF00080932001809321018093220180932301BB
:107000008093240180932501809326010E94C83338
:107010000E94521810E4C8E8D3E10E94B2292197D7
:10702000E1F780910201863711F40E9452180E9404
:107030003D3488B1812788B9EECFEE0FFF1F059050
:0A704000F491E02D0994F894FFCFBD
:02704A0037010C
:00000001FF
